:04000005000080C1B6
:020000040000FA
:10800000502800200983000011830000F59900002A
:10801000000000000000000000000000A137FEDFAB
:108020008F9E939B01999697FB000000B9810000F9
:1080300000000000000000005D820000BD82000022
:108040001B8300001B8300001B8300001B830000B8
:108050001B8300001B8300001B8300001B830000A8
:108060001B8300001B8300001B8300001B83000098
:108070001B8300000DA600001B8300001B83000073
:108080001B8300001B8300001B8300001B83000078
:108090001B8300001B8300001B8300001B83000068
:1080A000F5A600001B8300001B8300001B8300005B
:1080B0001B8300001B8300001B8300001B83000048
:1080C00000F002F800F030F80CA030C8083824188E
:1080D0002D18A246671EAB4654465D46AC4201D100
:1080E00000F022F87E460F3E0FCCB6460126334202
:1080F00000D0FB1AA246AB46334318471CCA000007
:108100003CCA00000023002400250026103A01D3B9
:1081100078C1FBD8520700D330C100D50B6070473F
:108120001FB51FBD10B510BD00F0F2FC1146FFF7E2
:10813000F7FF06F011FF00F00AFD03B4FFF7F2FFAE
:1081400003BC00F0BBFC000080F309887047EFF32C
:1081500009807047684680F3098806480078C007A0
:1081600003D1032080F314887047022080F3148821
:1081700070470000C4390100064B9C46EFF30583AD
:108180001B0605D1EFF31483DB0701D000DF704736
:108190006047000069FD0000064B9C46EFF3058335
:1081A0001B0605D1EFF31483DB0701D000DF704716
:1081B00060470000D9FF0000EFF309808169891E44
:1081C0000978002933D1A6461FC8A4467446E04763
:1081D0001F4B06CB914224D0083B002910D00CB491
:1081E000203101234B70EFF30983203B4B60F0C338
:1081F00044464D4656465F46F0C308F06BF90CBC4A
:108200001A60203253681033F0CBA046A946B2461C
:10821000BB4683F30988203BF0CB5078002803D07D
:108220001078EFF3098318600223DB43184710B579
:10823000084A1268914209D8074C89006458A6463A
:108240001FC8A446F047EFF309840FC410BD000017
:10825000D0F1FF1FF48B0000F48B000008F01CF835
:10826000154B06CB914223D0083B0CB420310023A0
:108270004B70EFF30983203B4B60F0C344464D46FF
:1082800056465F46F0C308F025F90CBC1A60203250
:1082900053681033F0CBA046A946B246BB4683F3E1
:1082A0000988203BF0CB5078002801D01078186165
:1082B0000223DB4318470000D0F1FF1F08F0DAF972
:1082C000CEE7000007F074F808F0D4F9C8E7000022
:1082D00070B505460C46164602E00FCC0FC5103EA1
:1082E000102EFAD2082E02D303CC03C5083E042E6A
:1082F00007D301CC01C5361F03E021782970641C27
:108300006D1C761EF9D270BD0748804707480047AC
:10831000FEE7FEE7FEE7FEE7FEE7FEE70448054965
:10832000054A064B704700005DA50000C1800000B3
:1083300050260020502800205027002050270020E1
:1083400000487047EC25002010B5002000F0BCFB71
:10835000FFF7E8FE012000F0B1FB10BD034610B5A9
:108360000B439B070FD1042A0DD308C810C9121F55
:10837000A342F8D018BA21BA884201D9012010BD11
:108380000020C04310BD002A03D0D30703D0521CE5
:1083900007E0002010BD03780C78401C491C1B1B13
:1083A00007D103780C78401C491C1B1B01D1921E7D
:1083B000F1D1184610BD000030B5441C03E001782F
:1083C000401C00290DD08107F9D10B4BDD0104C8F9
:1083D000D11A91432940FAD0001B0A0603D0C01ECF
:1083E00030BD001B30BD0A0401D0801E30BD090223
:1083F000FCD0401E30BD00000101010170477047F4
:10840000FFFFFFFFFFFFFFFFFFFFFFFFFEFFFFFF7D
:10841000FFB516460A46C3B0012141912092009053
:108420006A464198411E41918100091F80005558BC
:10843000001F20A9085842904010429970432C1800
:10844000C90700D1801B2146469A27182846904725
:1084500000280FDD314630462943890769D022784C
:108460002978401E2A702170641C6D1C0028F6D1EA
:10847000AD1BA41B3946469A20469047002825DDAF
:1084800039462846469A904700280FDD3146304647
:108490002943890755D03A782978401E2A703970C7
:1084A0006D1C7F1C0028F6D1AD1BBF1B314630462A
:1084B000214389074DD03A782178401E22703970C7
:1084C000641C7F1C0028F6D1A41BBF1B324631461A
:1084D0002243B81B920744D003782278491E2370A8
:1084E0000270401C641C0029F6D12C46871B409763
:1084F000469A4099A419204690470028F8DB469AEE
:108500004099BF1B384690470028F8DC304631467A
:10851000A74236D9214389072BD03A782178401ECB
:1085200022703970641C7F1C0028F6D1A41BBF1B6D
:10853000DEE722682968001F04C502C40028F8D1BC
:1085400096E73A682968001F04C502C70028F8D1D9
:10855000AAE73A682168001F04C402C70028F8D1BE
:10856000B2E703682268091F08C404C00029F8D1D3
:10857000BBE73A682168001F04C402C70028F8D18D
:10858000D4E72143890723D0409A2178401E1278EE
:108590002270409A641C11704099491C0028409137
:1085A000F2D13146A41B601B00F091F94299401EA4
:1085B000091A491E88421CDD0A2916DD6B46419ABC
:1085C00092009D5020AB98504198401C41901EE075
:1085D000409A2168001F126804C4409A11604099B3
:1085E000091D00284091F3D1DBE70A2813DD4290F2
:1085F00022E70A2809DD6B46419A92009C5020AB85
:1086000099504199491C4191F1E70A2903DD25461A
:108610000846429110E74198002800D000E747B093
:10862000F0BDFFB50E460746140081B03BD0002ECA
:1086300039D00A2E02D9049BFFF7EAFE761E3D468A
:108640006643701900902BE02E462D1900E0361B72
:10865000BE4205D329463046049A90470028F6DCEE
:1086600020462843311980070BD0002016E02A1835
:10867000136801E016681651121B8A42FAD2001DD7
:108680001351A0420CD2F2E72A18137801E01678B1
:108690001655121B8A42FAD2401C1355A042F3D33E
:1086A00000988542D0D305B0F0BD00000346F0B578
:1086B0000B439B072DD1244DEF01042A29D308C871
:1086C00010C95E1B9E43121F3E4017D0D8B2E1B2C4
:1086D000401A3106014310D198B2A1B2401A3104B8
:1086E00001430AD118022102000A090A401A310284
:1086F000014302D1180E210E401AF0BDA342DCD076
:1087000018BA21BA884201D90120F0BD0020C04327
:10871000F0BD002A01D10020F0BD03780C78401C88
:10872000491C002B0DD0A3420BD1521E09D0037857
:108730000C78401C491C002B03D0A34201D1521ECF
:10874000EBD1181BF0BD000001010101421E53785E
:10875000521C002BFBD10B78491C1370521C002BB0
:10876000F9D17047F8B5042A2CD3830712D00B78BF
:10877000491C0370401C521E83070BD00B78491C08
:108780000370401C521E830704D00B78491C0370F1
:10879000401C521E8B079B0F05D0C91ADF002023F7
:1087A000DE1B08C90AE0FFF793FDF8BD1D4608C9A6
:1087B000FD401C46B4402C4310C0121F042AF5D2C1
:1087C000F308C91A521EF0D40B78491C0370401CE0
:1087D000521EEAD40B78491C0370401C012AE4D4D1
:1087E00009780170F8BD431A70B593421BD28918FD
:1087F000801804E0491E401E0B78521E0370930738
:10880000F8D106E01039103878C9103978C010381E
:10881000103A102AF6D203E0091F001F0B6803600C
:10882000121FF9D570BDFFF753FD70BDF8B50646B0
:1088300014460843800707D0751AA54219D20819B3
:10884000102D13D2311907E03046FFF7CCFFF8BDE9
:10885000401E491E02780A70641EF9D2F8BD471BFB
:108860002A463946FFF77EFF641B3846A542F6D3F9
:10887000011B22463046FFF775FFF8BDD2B210B596
:1088800013029A1813049A1800F00EF810BD01E0B4
:1088900004C0091F0429FBD28B0701D50280801C6C
:1088A000C90700D00270704700290BD0C30702D05F
:1088B0000270401C491E022904D3830702D502809E
:1088C000801C891EE3E70022EEE70022DFE700229A
:1088D00003098B4273D3030A8B4258D3030B8B4299
:1088E0003CD3030C8B4221D312E003460B437FD4CD
:1088F000002243088B4274D303098B425FD3030ADF
:108900008B4244D3030B8B4228D3030C8B420DD3F1
:10891000FF22090212BA030C8B4202D3121209027F
:1089200065D0030B8B4219D300E0090AC30B8B42BD
:1089300001D3CB03C01A5241830B8B4201D38B036B
:10894000C01A5241430B8B4201D34B03C01A524110
:10895000030B8B4201D30B03C01A5241C30A8B4253
:1089600001D3CB02C01A5241830A8B4201D38B023E
:10897000C01A5241430A8B4201D34B02C01A5241E2
:10898000030A8B4201D30B02C01A5241CDD2C30954
:108990008B4201D3CB01C01A524183098B4201D3D0
:1089A0008B01C01A524143098B4201D34B01C01ABB
:1089B000524103098B4201D30B01C01A5241C30833
:1089C0008B4201D3CB00C01A524183088B4201D3A2
:1089D0008B00C01A524143088B4201D34B00C01A8E
:1089E0005241411A00D201465241104670475DE0A3
:1089F000CA0F00D04942031000D340425340002226
:108A00009C4603098B422DD3030A8B4212D3FC22CE
:108A1000890112BA030A8B420CD3890192118B424D
:108A200008D3890192118B4204D389013AD0921163
:108A300000E08909C3098B4201D3CB01C01A52411E
:108A400083098B4201D38B01C01A524143098B42E7
:108A500001D34B01C01A524103098B4201D30B01D0
:108A6000C01A5241C3088B4201D3CB00C01A5241F5
:108A700083088B4201D38B00C01A5241D9D24308DC
:108A80008B4201D34B00C01A5241411A00D2014619
:108A9000634652415B10104601D34042002B00D583
:108AA0004942704763465B1000D3404201B5002045
:108AB000C046C04602BD7047704770470149182044
:108AC000ABBEFEE72600020010B500F009F800F08A
:108AD00001F810BD10B5002801D0FFF7EFFF10BD61
:108AE00010B5002102A000F03AF8012010BD0000EE
:108AF000534947414252543A2041626E6F726D6150
:108B00006C207465726D696E6174696F6E0000002F
:108B10007546FFF715FCAE46050069465346C0088A
:108B2000C000854618B020B5FFF7F8FB60BC0027F1
:108B30004908B6460026C0C5C0C5C0C5C0C5C0C529
:108B4000C0C5C0C5C0C5403D49008D46704710B581
:108B50000446C046C0462046FFF7EFFA10BD70B588
:108B600005460C460A2000E06D1C00F012F8002DAE
:108B700006D028780028F7D102E0641C00F009F83C
:108B8000002C02D020780028F7D10A2000F001F84C
:108B900070BD08B5694608700320ABBE08BD70B54E
:108BA0008C180578401C6B075B0F01D10378401CC3
:108BB0002A1106D10278401C03E00678401C0E7092
:108BC000491C5B1EF9D12B0705D40023521E0DD47E
:108BD0000B70491CFAE70378401CCB1A921C03E087
:108BE0001D780D70491C5B1C521EF9D5A142D8D3CB
:108BF000002070BD00000000F8B502787F2A02D086
:108C000000F018F8F8BD0A704678851C4E708C1C70
:108C1000074F761E0AD32146284600F00BF8010CB8
:108C20003F1880B24D190419761EF4D23846F8BDAB
:108C300002000200F0B5027885B01346803B1F2B7E
:108C400003D800F0BFFA05B0F0BD0A704E1C0178E1
:108C5000401C17297CD20A007A4412799218974452
:108C60000B3B4865FEFDFC77FB788077777777775D
:108C700085FAF9F8F7F6F50000780021062826D0E5
:108C800009DC052823D202007A441279921897440D
:108C90001E1E1E1E0B00F0280CD0FD2817D0FE282B
:108CA00012D0FF2813D109E0F749701C04F0CBFA69
:108CB00005210CE011207070012108E04020707047
:108CC0000020B070022102E0052070700121EF4801
:108CD0003170081805B0F0BD0078002805D00128D3
:108CE00003D0FF203070EA4841E200203070E848AD
:108CF0003DE20078002805D0012804D00020307023
:108D0000E44834E20120E44A01211170E3492024BF
:108D10004C6040224A604A604B6923434B614B6977
:108D200013434B614B6913434B61E8E7DA48002377
:108D30000370DA4841692022914341614169402230
:108D400091434161416991434161337001200EE2D9
:108D50002AE241780278080210430001401EFDD14A
:108D6000C3E7002070703070022000E2831C1C46B4
:108D7000257802782B46657841782D022B43A5781B
:108D8000E4782D042B432406234340791B021B0A5D
:108D900000060343C80708D0D00703D0BF4C2020EB
:108DA000606002E0BD4C2020A060880708D59007D5
:108DB00003D5BA4C4020606002E0B84C4020A0606F
:108DC000080609D5D009C00703D0B44C4020606024
:108DD00002E0B24C4020A060002B31D0B04883426A
:108DE00000D90346AF4C0025A561302043436361A1
:108DF000052020615308A94FD009CD0704D03D6953
:108E0000AD06ED0F954215D18D0704D53D696D0670
:108E1000ED0F9D420ED14D0701D595080AD18D0663
:108E200001D5550906D10D0608D53D696D06ED0F32
:108E3000854203D02569ED03ED0FDED000202061CF
:108E4000964A106911698006C00F09E083E07BE053
:108E500062E054E041E00FE082E1AFE090E07EE0CC
:108E60004906C90F4900084311694906C90FC901DC
:108E7000084330708C487AE10378C2781946437809
:108E800012061B0219438378C0781B04194311434F
:108E90000902090A0006014307D08448814208D329
:108EA0007D4901204870486013E0FF203070804801
:108EB0005DE1794C002060707E480818FFF707FDDF
:108EC000012804D90321401CFFF701FD00E0012027
:108ED000606000203070764849E10478401C002C26
:108EE00001D1FF2401340146204601F00FFB002090
:108EF0003070E41DE00867490004401837E100784D
:108F000065498207920F521C40070A75C00F4875C9
:108F1000002030705F482AE1FF2131700122037880
:108F2000401C14465B1E0CD30178401C8906890E38
:108F300000D14021C91DC90852184018521C5B1E9F
:108F4000F2D21004204312E10078FF213170514920
:108F5000000440180BE1FF2030704E4807E14E4AF4
:108F60000178117283784478190221435181017983
:108F7000C378080218439081002030704E48F6E014
:108F8000454A31461278012A15D00446401C027821
:108F9000401C002A08D00378401C9D0701D5DB0641
:108FA00000D5001D521EF6D10022001B0A700004DD
:108FB0007270801CDBE000F0A5F9D8E00390364821
:108FC000007801280CD0002030707070B070032041
:108FD0000399C978890756D5012189040843C6E059
:108FE00000243649039D029620460C70A9786A78C1
:108FF0000F021743ED1CF61C002F43D029786D1C7F
:10900000009189075CD50099C90711D0224845898C
:109010000021009801F000F8022802D0012831D187
:1090200006E06D1E2ED3254909780029F0D082E094
:109030007F1E27D3002F04D10098C00701D00E2037
:1090400000901548458901A9009800F0E5FF022825
:1090500002D001286FD106E06D1E6CD31749097844
:109060000029F0D067E0019931700199641C090A68
:1090700071700199090CB1700199090EF170361DDA
:109080007F1ED7D257E060E01839010002000200CD
:10909000010002000100010018F3FF1F80F00F40E3
:1090A000C0C62D0000E000E00100060000366E01A1
:1090B00001000400FF356E010100050004F0FF1FF0
:1090C0007F1E04972A78E97810466A78090612020A
:1090D0001043AA78120410430843E9780002000AFA
:1090E00009060843019033482D1D478901A90098BE
:1090F00000F092FF022802D001281CD106E07F1E5A
:1091000019D32D4909780029F0D014E00498641C83
:10911000401E0490401C0028D4D12648264F458983
:1091200000210E2000F078FF022804D16D1E02D32A
:1091300039780029F4D002990C70029A210A5170F2
:10914000029988700298301A42E703998A784B781E
:10915000110219430122890492048918084306E088
:1091600014490978012906D0FF20307013481449AA
:1091700005B04018F0BD411C0A4613780079194625
:10918000537800061B0219439378D2781B041943C5
:10919000120611430902090A0143009169460020A1
:1091A00000F03AFF0020E0E7FF20203EF07704487F
:1091B00005B0F0BD18F3FF1F04F0FF1F010005000C
:1091C00001000100F0B583B002780A704D1C0178EF
:1091D000474C461C80390D2943D208007844007959
:1091E0000018874406141F3F4781818153616C72C8
:1091F000770005F09FFD0746FFF7DEF8C6B22E7038
:10920000681C32463946FFF7ADFAA41930E007244E
:10921000684601F035FC224669462846FFF7A2FA67
:10922000344C61E0684601F02BFC3178FF2208469F
:10923000717812020902904311400843B17812027A
:109240000904904311400843F1780906084300904F
:10925000684601F037FC002001F0BCFC01202870BA
:10926000254C41E03E21681C08F0A0FD2870241820
:10927000641C39E03778701C394608F005FE01207F
:10928000287038041A49001944182DE0012028706C
:109290003078002805D0012803D000202870174C12
:1092A00022E006F021F8FAE70120287004F020FA05
:1092B000002802D1022008F0E9FB114C14E03078BC
:1092C00007F0F2FC28700D4C0EE007F0ABFC2870A4
:1092D0000B4C09E03778701C394607F065FD2870A3
:1092E0003804034900194418204603B0F0BD0000BB
:1092F0000100010009000100020005000200020057
:1093000002000100F0B589B00890044600208D1CD1
:109310000391C04902900870049005906778A41CDE
:10932000002F6FD02178641C019189076BD50499B7
:1093300000292FD0B84811214689019808400128FA
:109340000CD16946019800F067FE022814D1761E00
:109350004CD3B04909780029F3D008E169460E20C2
:1093600000F05AFE022805D1761E03D3A9490978D8
:109370000029F3D000210491012837D100992970E8
:109380000099090A69700099090CA9700099090EE1
:10939000E9702D1D0199C90659D52278E17810464A
:1093A0006278090612021043A2781204104308439F
:1093B000E1780002000A0906084307909648241D38
:1093C000808906900198C00711D0934846890021F2
:1093D000019800F021FE022802D0012806D106E003
:1093E000761E03D38B4909780029F0D0BFE08A4864
:1093F00046896946019800F00FFE022804D0012832
:1094000019D108E0F8E05BE0761E14D381490978B1
:109410000029EED00FE08049009A09691140079AAF
:10942000914208D00699491E0691491C03D07949FA
:1094300009780029DBD07849009A09691140079A18
:10944000914201D01021084301284DD136E07249E4
:109450004E890199C90715D0049900292ED1002100
:10946000019800F0D9FD022802D001287FD106E042
:10947000761E7CD3674909780029F0D077E0012176
:1094800004911BE06946019800F0C6FD022802D055
:1094900001286CD106E0761E69D35E49097800295F
:1094A000F0D064E0009929700099090A6970009968
:1094B000090CA9700099090EE9702D1D00214EE0DC
:1094C000049800281FD05448468969460E2000F0B1
:1094D000A3FD022802D0012849D106E0761E46D31A
:1094E0004C4909780029F0D041E000982870009894
:1094F000000A68700098000CA8700098000EE870D0
:1095000000202D1D04902278E1781046627809062B
:1095100012021043A278120410430843E1780002BB
:10952000000A090608430199241D0090890603D505
:1095300039490861012013E0374846896946019896
:1095400000F06AFD022802D0012810D106E0761E44
:109550000DD3304909780029F0D008E001210591A8
:109560000299491C02912B49097800290DD0002F3E
:1095700008D02178641C8A0701D5C90600D5241DAE
:109580007F1EF6D1012804D036E07F1E00D0C9E648
:10959000F8E7049900291ED01F481E4F46896946E6
:1095A0000E2000F039FD022802D0012824D105E068
:1095B000761E21D339780029F1D01DE00099297059
:1095C0000099090A69700099090CA9700099090E9F
:1095D000E9702D1D10E0059900290DD00E480D4FA2
:1095E000468900210E2000F017FD022804D1761EC6
:1095F00002D339780029F4D0039A029911700399A3
:10960000487008980399201A0004691A084309B0A1
:10961000F0BD000004F0FF1F18F3FF1F10B4164840
:109620000021017041700322426001726422428174
:10963000818101220161027541751048816B1F22F1
:10964000520211438163FF200D4B033058610D48D6
:109650002021416042690A434261FF2404349C6135
:109660004021416042698A4342619C614160426994
:109670000A43426110BC704718F3FF1F008004408A
:1096800000B0044080F00F4070B50546EFF3108045
:10969000C407E40F72B6094E094B29463046F268FA
:1096A00000F010F8002805D1002329463046F26862
:1096B00000F010F9002C00D162B670BD50160020E9
:1096C0006B66656BFFB589B015460C466A4609980E
:1096D00005F090F82A462146049B099804F035FECF
:1096E000070030D1009C019E65196D1E3146284649
:1096F000FFF7EDF8002902D0401C7043451EAC4234
:109700001DD821020920090A000609180F484160E6
:109710000F490C98884201D06B2000E000200028FF
:1097200011D1099804F02CFE074609980069002819
:1097300000D08047002F02D1A419AC42E1D909988A
:1097400004F0DAFD38460DB0F0BD00000000024024
:109750006B66656B002801D10420704770B5044624
:109760001548C0680001000F0F2821D013494000A0
:10977000085A80020025256060600120A0606561B4
:10978000A56180022561E060E069002802D00068E0
:10979000022809D00A480B49056041600A498160E6
:1097A000E061204600F012F825620020656270BD7D
:1097B00001204004DEE70000408004402C3E010010
:1097C0000417002084160020C4160020002801D1B0
:1097D0000420704770B5C4691548402241081548F7
:1097E0004900400840006568884202D9421A402A70
:1097F00012D82846FEF7B6FF10480F4E4108104811
:109800006D1C35604008402249004000A568884230
:1098100004D9421A402A01D9FEF796FD2846FEF7E0
:10982000A1FF6D1C022075602060002070BD00004B
:10983000F1EA0000FDEA000048F1FF1F35E30000F7
:1098400049E30000002A01D104207047FFB589B028
:1098500014461E460D466A46099804F0CBFF324670
:109860002946039B099804F070FD07002DD1009D47
:10987000002E26D002CC164881600399042902D01C
:10988000082907D00EE02A020321120A49065118BE
:10989000416007E002CCC1602A020721120A0906D2
:1098A00051184160099804F06BFD0746099800695A
:1098B000002800D08047002F03D103984519361A9D
:1098C000D8D1099804F018FD38460DB0F0BD00005D
:1098D00000000240FFB58BB014461E460D466A4696
:1098E0000B9804F087FF22462946059B0B9804F04D
:1098F0002CFD002833D16A4629460B9804F07AFFE4
:10990000009D029808906942404201404F42AF4298
:1099100001D108983F18002C20D0300209907E1BFE
:10992000A64200D9264630460599FEF7D0FF2A0206
:109930000121120A090652180A494A60099A0004CC
:109940001043FF3088600B9804F01AFD002806D100
:109950000898A41BAD193F18002CE0D100200FB0CF
:10996000F0BD000000000240002B01D10420704730
:10997000FFB589B016461D460C466A46129F0998E7
:1099800004F038FF32462146079B099804F0DDFCBD
:1099900000281DD1009C002E1AD014493806471803
:1099A00021020120090A4006091811484160876018
:1099B0002968C160099804F0E3FC00280AD01399D3
:1099C000002900D00C601499002901D000220A60FF
:1099D0000DB0F0BD0799761A890889004D190799CD
:1099E0000C19002EDCD10DB0F0BD0000FFFFFF0010
:1099F00000000240EFF3088470460007000F0D28B6
:109A000001D1EFF309842546A08B2035800500D5D0
:109A10002D1D7046C00600D44835704603F0E0FEA8
:109A2000EFF3098003F0DCFEEFF3088003F0D8FECB
:109A3000EFF3148003F0D4FE284603F0D1FE6069F2
:109A400003F0CEFEA06903F0CBFEE06903F0C8FE90
:109A500000F0D0FDFEE770B5044600F057F800F0C6
:109A600049FA07F059F8162007F094F8FF2007F09C
:109A700091F8054607F04AF807F04EF82806250C3D
:109A8000002809DA202007F085F8284607F0A6F814
:109A9000A0B207F0A3F808E00121E8B2490340189A
:109AA00007F09CF8A0B207F099F807F02FF870BD06
:109AB00010B5002000F0D7F80B4C53280ED1012030
:109AC00000F0D1F8462809D1022000F0CCF8442853
:109AD00004D1032000F0C7F8502803D000202070E4
:109AE000C0B210BD0120FAE7C0F1FF1F10B5054953
:109AF0000020087007F016F80348012181604160DA
:109B000010BD0000C0F1FF1F40F00F4010B507F07E
:109B100003F8052007F03EF8FF2007F03BF8044665
:109B200006F0F4FFE007F2D110BD00000148007814
:109B300070470000C0F1FF1FF8B517460C460646F7
:109B400006F0EAFF052007F025F8FF2007F022F8CD
:109B5000054606F0DBFFE807F2D106F0DDFF062040
:109B600007F018F806F0D2FF06F0D6FF052007F040
:109B700011F8FF2007F00EF8054606F0C7FFA8070A
:109B8000F2D5FF20E1B20130451AAF4200D83D4680
:109B900006F0C2FF162006F0FDFFFF2006F0FAFFD8
:109BA000009006F0B3FF06F0B7FF0098000609D555
:109BB000022006F0EFFF200C07F010F8A0B207F02B
:109BC0000DF809E02002000EFF30FF30023007F0F0
:109BD00005F8A0B207F002F864197F1B3078761CF4
:109BE00006F0D8FF6D1EF9D106F090FF002FA7D127
:109BF000F8BDF8B515460E460746FFF787FF06F095
:109C00008BFF162006F0C6FFFF2006F0C3FF0446B8
:109C100006F07CFF06F080FF200609D5032006F041
:109C2000B9FF300C06F0DAFFB0B206F0D7FF09E05A
:109C30003002010E03200002081806F0CFFFB0B278
:109C400006F0CCFF0024002D06D9FF2006F0A2FF6D
:109C50003855641CAC42F8D306F058FF7F197619CA
:109C60006D1BCCD1F8BD10B5044606F055FF5A2047
:109C700006F090FF002006F08DFF002006F08AFF1E
:109C8000204606F087FFFF2006F084FFFF2006F045
:109C900081FF044606F03AFF204610BDF7B584B0B8
:109CA0000020009006980C0B08180D462403029023
:109CB0008C49001B4018000B019070D08A4801218C
:109CC00040680906884252D3FF2087490004486053
:109CD000FFF71CFF00F00EF906F01EFF162006F03D
:109CE00059FFFF2006F056FF064606F00FFF06F06C
:109CF00013FF300609D5D82006F04CFFFF2006F0F0
:109D00006DFF002006F06AFF05E0784806F066FF68
:109D1000002006F063FF06F0F9FE0120000326187C
:109D20002746B44279D2F81DF9300390A84276D97B
:109D30000399029888423DD3AF4231D2FF220132CB
:109D400039466B48FFF755FF69487A1BE91B08182D
:109D5000FF3201320499FEF705FD6348391B406864
:109D6000FF22091801326248FFF7E6FE66E0FF2194
:109D700009048842D1D1FFF7C9FE00F0BBF806F014
:109D8000CBFE162006F006FFFF2006F003FF064676
:109D900006F0BCFE06F0C0FE3006B6D5ABE79EE08E
:109DA0005148391B40687A1B091804981018FF2283
:109DB00001322FE0AF4216D2FF22013239464C4821
:109DC000FFF717FF4A48E91B0818069A0499FEF79F
:109DD000C9FC4548391B4068FF2209180132444834
:109DE000FFF7AAFE2AE0B84219D9FF22013239460C
:109DF0003F48FFF7FEFE0298791BC21B0498091822
:109E00003B48FEF7AFFC3848391B4068FF22091871
:109E100001323748FFF790FE10E013E0FFE7FF2222
:109E2000013239463248FFF7E4FE2F48391B4068BB
:109E3000FF22091801322E48FFF77EFE039FB7422A
:109E400000D270E7FFF762FE00F054F806F064FEFF
:109E5000162006F09FFEFF2006F09CFE074606F047
:109E600055FE06F059FE380609D5202006F092FE70
:109E7000200C06F0B3FEA0B206F0B0FE09E020020E
:109E8000010E01204003081806F0A8FEA0B206F05B
:109E9000A5FE06F03BFE2746B44212D21248391BFB
:109EA0004068FF22091801321148FFF7A2FEFF2285
:109EB000013239460E48FFF73FFEFF370137B74200
:109EC000ECD3094801214268090351184160009808
:109ED0000199401C34460090884200D2EEE607B05B
:109EE000F0BD0000FF0F0000C0F1FF1FFFD8000011
:109EF000B523002010B506F00FFE062006F04AFE3E
:109F000006F004FE06F008FE052006F043FEFF20E2
:109F100006F040FE044606F0F9FDA007F2D510BD9C
:109F200070B5064615460C46080503D03046FFF7C7
:109F300003FE70BD0846FFF78EFD2A4621463046D7
:109F4000FFF7FAFD70BD000010B5EFF31080C007F9
:109F5000C00F72B60021064A1160002800D162B617
:109F60000448FFF7F7FB002800D0012010BD0000D7
:109F7000008104405016002010B582B000206946D0
:109F8000FF240C54401CC0B20828FAD3332000F040
:109F9000BDFA9E2069460870E7204870102000F046
:109FA000B5FA002069460C54401CC0B20828FAD308
:109FB000332000F0ABFA002069460870082000F05A
:109FC000A5FA01A9002007F0FDF8012800D0002023
:109FD00002B010BDF0B583B0074616460D46EFF34C
:109FE0001080C407E40F72B60B4639460948FFF7E4
:109FF00029FC002809D101210190009102903346EB
:10A000002A4639460348FFF7AFFC002C00D162B660
:10A0100003B0F0BD5016002000B5054A5278002A62
:10A0200002D000F007F800BD00F0E8F800BD000025
:10A0300018F3FF1FF0B402466E4E402070602027D8
:10A04000B7607760D30701D0706000E0B060B760A0
:10A0500077605308DD0701D0706000E0B060B76042
:10A060007760D4189308DD0701D0706000E0B0601D
:10A07000B7607760E418D308DD0701D0706000E0B6
:10A08000B060B7607760E318DB0701D0706000E074
:10A09000B060B7607760B060B76077607060B760DD
:10A0A000776073694020834373615348007D031ECA
:10A0B00003D0B7607760401EFBD1B760306977602E
:10A0C0004006C00FB760346977606406E40F64002F
:10A0D0000443B760306977604006C00F80002043BA
:10A0E000012810D0022862D0042860D0213303D088
:10A0F000B76077605B1EFBD1726940210A437261D1
:10A100007160F0BC7047920726D500231C462022C0
:10A11000B760356977606D06ED0F64195B08ED0770
:10A120002B43521EF4D1B760326977605206D20FCA
:10A130005440E20700D00820002900D00B602E49CF
:10A14000097D002903D0B7607760491EFBD1716992
:10A150004022114371611EE0002B03D0B76077608D
:10A160005B1EFBD1726940252A4372610968002396
:10A170002022CC0701D0756000E0B560B760776041
:10A180005B184908521EF4D1D90701D0756000E070
:10A19000B560B76077601849097A002905D0402278
:10A1A000B260B7607760491EFBD14021A8E7124931
:10A1B0004C7D002C06D0910704D52121B760776033
:10A1C000491EFBD1002B03D0B76077605B1EFBD12B
:10A1D0007169402319437161002C07D0910705D4A0
:10A1E000B3602121B7607760491EFBD17360F0BC7A
:10A1F0007047000080F00F4018F3FF1FF0B58C4649
:10A2000004460020BF4940234B6020268E60BE4F8D
:10A210007A6815466D1EFDD14E6015466D1EFDD146
:10A22000E50701D04B6000E08B608E6015466D1E27
:10A23000FDD14E6015466D1EFDD105196008C7079A
:10A2400001D04B6000E08B608E6017467F1EFDD111
:10A250004E6017467F1EFDD12D18A008C70701D0FC
:10A260004B6000E08B608E6017467F1EFDD14E6014
:10A2700017467F1EFDD12F18E508E80701D04B6077
:10A2800000E08B608E601046401EFDD14E6010468F
:10A29000401EFDD17819C00701D04B6000E08B60F3
:10A2A0008E60994D1046401EFDD14E601046401EF6
:10A2B000FDD18B608E601046401EFDD14E60104671
:10A2C000401EFDD14B608E601046401EFDD14E6099
:10A2D0001046401EFDD148694023984348612B7DBC
:10A2E0001D1E09D08E601046401EFDD14E601046E6
:10A2F000401EFDD15B1EF5D18E601046401EFDD183
:10A3000008694E604006C00F13465B1EFDD18E608B
:10A3100013465B1EFDD10B694E605B06DB0F1746D3
:10A320007F1EFDD15B0003438E601046401EFDD1B1
:10A3300008694006C00F20264E601646761EFDD1E5
:10A3400080001843012816D002286ED004286CD053
:10A3500021350AD020248C6013465B1EFDD14C6051
:10A3600013465B1EFDD16D1EF5D14A6940231A4389
:10A370004A614B60F0BDA3073CD500252E46202442
:10A3800020238B6017467F1EFDD10F694B607F062F
:10A39000FF0F13465B1EFDD16B08FD07F6191D4329
:10A3A000641EEDD120238B601446641EFDD10C6920
:10A3B0000F466406E40F4B60521EFDD16640F20763
:10A3C00000D008206246002A00D015604E4A147D55
:10A3D000002C0AD05568BB602A46521EFDD17B6016
:10A3E0002A46521EFDD1641EF5D17B6940221343DB
:10A3F0007B6139E0002D0AD020248C6013465B1E5F
:10A40000FDD14C6013465B1EFDD16D1EF5D14C692C
:10A4100040231C434C6164460026246820252F46B7
:10A42000E30703D040234B6002E032E040238B601F
:10A430008F6013465B1EFDD14F6013465B1EFDD13E
:10A44000361964086D1EEBD1F30702D040234B6030
:10A4500001E040238B603C460D468F6013465B1E37
:10A46000FDD16C60521EFDD1274A137A002B0DD00E
:10A4700040248C60546820258D602246521EFDD1F8
:10A480004D602246521EFDD15B1EF5D140224A602E
:10A49000F0BD1D4B5B7D9C46002B0DD0A3070BD55B
:10A4A000212620278F6013465B1EFDD14F60134687
:10A4B0005B1EFDD1761EF5D1002D0AD020268E60C0
:10A4C00013465B1EFDD14E6013465B1EFDD16D1E13
:10A4D000F5D14B6940252B434B616346002B0ED0D1
:10A4E000A3070CD48D60212420268E6013465B1EAA
:10A4F000FDD14E6013465B1EFDD1641EF5D14D604B
:10A50000F0BD000080F00F4018F3FF1FF0B4124CB4
:10A51000104E20276568401E03D2F0BC7047002B08
:10A5200002D10C780823491CE20702D04022726055
:10A5300001E04022B260B7602A46521EFDD177602A
:10A540002A46521EFDD164085B1E401EE7D2F0BCB5
:10A550007047000080F00F4018F3FF1F1D480022D5
:10A5600002601D48816B4315194381631C491B48D8
:10A5700048601C4883681C490B408360C3680B40DB
:10A58000C3601A4980200870194824214170A22113
:10A590000170C178C906C90EC170032101714271F1
:10A5A0008179C906FCD481790907890F0229FAD17A
:10A5B0004021417181790907890F0229FAD18179F6
:10A5C0004906FCD51A21017081790907890F0329F1
:10A5D000FAD170470081044000800440000001105F
:10A5E0004080044040900440FFF8FFFE00500640C9
:10A5F00000400640BFF34F8F03490248C860BFF3D5
:10A600004F8FFEE70400FA0500ED00E038B5254D58
:10A610002C79E878800601D420208443E87800066D
:10A6200001D480208443200616D51F4802F0F4FE92
:10A63000002800D00120E7221CA102F053FE1A4896
:10A6400002F00AFFE871184802F0E6FE002803D184
:10A65000E8784006400EE870A00605D56007800F38
:10A6600003D0E8796946087038BDED791B4802F0DF
:10A67000B5FE0446132804D92946184802F018FFED
:10A6800038BD03F045F8002807D0132CF8D1132269
:10A6900013A1124802F094FF38BD104802F0DCFE0E
:10A6A000EAE7000000B00640101700202E2E5C2EB6
:10A6B0002E5C2E2E5C736F757263655C6869635FD8
:10A6C00068616C5C667265657363616C655C6B6C1C
:10A6D00032367A5C756172742E6300002019002096
:10A6E0003C4441504C696E6B3A4F766572666C6FB4
:10A6F000773E0A00F8B5314E00243078009001070B
:10A7000041D5317C0A090807C00F4B07DB0F1546FE
:10A7100005431AD1950040002818C018284FC000E2
:10A720003B5C9B061B0F012B0FD1C3195D88002DCD
:10A730000BD1244DAA5C5A803A5C520601D588227E
:10A7400000E0C8223A5401200143EFF31080C5070E
:10A75000ED0F72B61C4A1D4FB86811541521401CEC
:10A76000FEF7B5F8B960002D00D162B60820307050
:10A77000002C02D1307D800601D5012400E00024A8
:10A7800030780107BDD4009A0243EFF31081C90766
:10A79000C90F72B60E4B1D6815431D60002900D10C
:10A7A00062B6002C01D0012100E00021074A137895
:10A7B00019431170307002F0F7FCF8BD802007409B
:10A7C000001E0020B8F1FF1FA0230020A4F1FF1FEE
:10A7D000B0F1FF1F0020704770B50B4D0C460346CB
:10A7E000696B286B88420BD9401A844200DD04460D
:10A7F00022461846FDF7B6FF686B0019686300E053
:10A800000024204670BD00004CF2FF1F002070475E
:10A81000F8B5184F0C46064679693869401A16494A
:10A820000988081A002801DC0020F8BD844200DDF8
:10A830000446FA69B869002590420DD30F4A0319FE
:10A8400051188B4208D30D1A2A463146FDF78AFF6C
:10A8500076190A48641BB861002C06D0224631469E
:10A86000FDF780FFB8690019B861396960190918E6
:10A870003961F8BD4CF2FF1F723E0100321C00200E
:10A88000F8B5234CA06800283DD0616920690026F6
:10A89000421AE06811460143002935D021461D4F78
:10A8A000C9691D4D002A10D0A069814205D338889E
:10A8B0008B182818834200D3421A184800784300A6
:10A8C0001748C05A904200DA02461648E6600078FF
:10A8D0008023184302F07AFCE1690918E16162699A
:10A8E000121862613B88EB188B4200D1E561216947
:10A8F00091420BD1094909784A000949895A814294
:10A9000004D10120E060F8BDA660F8BDE660F8BDA6
:10A910004CF2FF1F723E0100321C00208FF2FF1F1D
:10A92000763E0100703E010010B50C4C206A0028F4
:10A9300003D0A06A401CA06210BD012020626062AA
:10A9400000F00EF8002060622062616B206B88428C
:10A95000F2D0401AFFF75AFF10BD00004CF2FF1F63
:10A9600010B5134C1348216B154B0A1A1248008876
:10A97000821A124800784000185A82420EDB1148B1
:10A98000007802F015FA216B08182063A06A0028ED
:10A990000CD0616A002909D1401E06E00120E06266
:10A9A000606A002802D0A06A401CA06210BD0000AE
:10A9B0004CF2FF1F721C0020743E01008FF2FF1F3B
:10A9C000763E0100713E010010B50446400702D5F5
:10A9D0002046FFF7A9FF200709D5054C606800282D
:10A9E00005D101206060FFF74BFF0020606010BDC3
:10A9F0004CF2FF1F002070470020704710B50B4835
:10AA000000F03EF8002810D0084A09491068087084
:10AA1000030A4B70030C8B70000EC870107908711C
:10AA20005079487190798871012010BD84F2FF1F20
:10AA3000301B002010B50E48002141608160C160CC
:10AA400001610C4A82614161016241628162C261BD
:10AA5000C162094A026342630180E122074852024F
:10AA60000260017141710821817100F01DF810BD73
:10AA70004CF2FF1F321C0020721C002084F2FF1FCA
:10AA8000084A116801700B0A43700B0C8370090EA1
:10AA9000C1701179817151794171917901710120F0
:10AAA0007047000010F3FF1F10B507F045F904F0E0
:10AAB00087FA012010BD10B507F082F9012010BD02
:10AAC0000120704710B50378C27819464378120602
:10AAD0001B02194383781B0419431143064A116072
:10AAE0008179117141795171007990710020D07193
:10AAF000104607F07BF910BD10F3FF1F10B50F488B
:10AB0000002444608460C46004610D498161446133
:10AB1000046244628462C462C1610A4901634163A0
:10AB20000480FFF7C8FFE121074849020160047172
:10AB3000447108218171FFF7C5FF10BD4CF2FF1F62
:10AB4000321C0020721C002084F2FF1F10B5FFF79A
:10AB5000D5FF10BD1C480078002833D070B51B4CC1
:10AB60000025206A012600280AD1616B206B8842EB
:10AB700006D11749884203D02163E56225626163EB
:10AB8000A06A002810D0206A00280DD1E06A0028B1
:10AB90000AD12662FFF7E4FE2562616B206B8842D2
:10ABA00002D0401AFFF732FEA1686068084308D15E
:10ABB00061692069884204D06660A660FFF760FE84
:10ABC000656070BD704700008DF2FF1F4CF2FF1FE3
:10ABD000721C0020B0B505460F480068C16988475F
:10ABE000002817D10D4C0E4F002D06D0BC4600DFBB
:10ABF0002060002006F04AFF0CE0BC4600DF216820
:10AC0000401AFF212D31884201D3012000E00020AD
:10AC100004F0E4F90120B0BDFC3901000CF3FF1F82
:10AC2000B1060100002070470020704710B50249AE
:10AC30000880FFF745FF10BD4CF2FF1F10B50E4B0B
:10AC40001A78D97810465A780906120210439A7871
:10AC50001204104308430102D878090A0006014390
:10AC600006480160197901715979417199798171A9
:10AC7000FFF728FF10BD0000301B002084F2FF1FEB
:10AC800001078A0E044900B551180A78FD231A40BD
:10AC90000A7002F021FA00BDC020074000B501464D
:10ACA0004A790B79807811021943020601D4024ACD
:10ACB000115402F011FA00BDB8F1FF1F704710B532
:10ACC00000F0D4FD10BD000008490028084A087DA6
:10ACD00004D0012318430875102005E04008400007
:10ACE0000875107AEF2108401072704780200740E5
:10ACF0000021074010B50B4C0B48A2880078824217
:10AD000000D90246002A02D108490020087180209B
:10AD1000216802F05BFA216809182160A188081AED
:10AD2000A08010BDA0F2FF1F503E01008CF2FF1F5B
:10AD3000704700000849020607D50007800E40183A
:10AD40000178FA22114001707047800040180178A4
:10AD5000F622114001707047C020074008490206E2
:10AD600007D50007800E40180178052211430170B5
:10AD70007047800040180178092211430170704724
:10AD8000C0200740F1B584B0049880076FD5082231
:10AD9000F849002002F00CF8F64C2078C009FFF7C3
:10ADA000C7FFF548E188818020784106890F04D0EB
:10ADB00001297DD002297CD1EFE2EE4949780C29A6
:10ADC00077D20A007A441279921897440542725158
:10ADD00072607772F4F3F2F1E649C006C00E04D057
:10ADE000012806D0022864D112E0E348E34901605B
:10ADF00026E1E3484278002A5BD0097980788142D5
:10AE000057D2E048002101704170DB49086017E12A
:10AE100008798F210840010605D50207120F01218C
:10AE20000904914001E001218140D54A5378002B6B
:10AE300001D100073DD1906808423AD0D06808405F
:10AE400000D00120CF490870000A4870CA4801604C
:10AE5000F6E0002002F0A4F800282AD000221146D3
:10AE6000802002F0B3F9C848006800287AD1AEE229
:10AE7000012002F095F800281BD000221146802006
:10AE800002F0A4F9C048006800286BD19FE2B949DC
:10AE9000C006C00E0DD1887880210843B8490870DB
:10AEA0004006400E012102F069F90022114601E03E
:10AEB00061E27CE0802002F089F988E2AD4BC006B7
:10AEC000C00E02D0012872D1A5E0D878062812D091
:10AED00006DC012809D002281ED0032867D16DE0C6
:10AEE000072844D00F2862D185E0A348A749016014
:10AEF0001220019095E0A6480078002857D0A0487D
:10AF0000C078002804D09C48A24901600A202CE0A7
:10AF10009948A1490160F9E79D480078002803D1CC
:10AF20009748C078012842D09548C07800281AD0A8
:10AF30009A4800909B780020002B0CD000990A784A
:10AF4000002A05D0CA788C78120222435118009149
:10AF5000401C8342F2D100980178002927D086490D
:10AF6000086053E0CAE18E48E3E7019059E0884861
:10AF7000007800281BD08248C07800281CD089485F
:10AF800000909B780020002B0CD000990A78002AB2
:10AF900005D0CA788C781202224351180091401CC7
:10AFA0008342F2D100980178002900D0D7E799E0D8
:10AFB00051E13CE150E046E07B48E1E77B4800900E
:10AFC0009978032914D00020002909D000990A7823
:10AFD000002A01D0511800919978401C8142F5D186
:10AFE0000098017800297DD0634908600078BCE7AB
:10AFF00003F0A4FEF8E76E480078002872D06D4890
:10B000005D4900900860017800296BD0C178827892
:10B0100008021043A9E701A9684601F073FF002860
:10B0200060D0554901988A88824209D980B28880C7
:10B0300061490978491E084202D151480121017134
:10B04000FFF758FEC3E1C006C00E4BD14A485B492A
:10B050000160FFF74FFEBAE10021C0060091C00E6B
:10B0600040D14448807800286FD0494800780028B3
:10B0700003D14348C078012834D0414EF0780028ED
:10B080000CD0464C2078002873D001276078022825
:10B0900006D0042848D0052866D148E0404CF1E7A6
:10B0A000344861798078814239D17070207944497F
:10B0B000B0700B880020002B05D9424A00211154A2
:10B0C000401C9842FBD301253846B168A84008428D
:10B0D00002D02846FFF72EFE01200004B168A840E8
:10B0E000084200E009E104D0284680210843FFF728
:10B0F00021FE6D1C102DE7D33348B0600020F060B6
:10B10000306135460120FFF7D9FDE0794006E88837
:10B1100001D5384301E040084000E88024E0E078B1
:10B12000A1780002084320E0E07800901CE000983D
:10B13000002819D1A5788F200540280606D52907B3
:10B14000090F01200004884002E03FE03846A84093
:10B15000B16801432046B160FFF7A0FD2846FFF724
:10B16000FDFD284601F0B8FF20780419207800285A
:10B170008CD14CE0A8F2FF1FA0F2FF1F92F2FF1F3C
:10B180008CF2FF1F301B0020D83E0100023F01005F
:10B190004B3E0100153F0100143F010085400100B6
:10B1A000F93F01008740010086400100884001000E
:10B1B0004C3E0100C03F0100503E01008DF2FF1FD8
:10B1C0004E3E010097F1FF1F010001000026AF4D28
:10B1D00001246E7080270120A968A040084202D097
:10B1E0002046FFF7A7FD01200004A968A0400842FF
:10B1F00003D020463843FFF79DFD641C102CEAD392
:10B20000EE60A3482E61A8600020FFF757FDA1481B
:10B2100081781C38407881426FD10022114680200D
:10B2200001F0D4FF9C480068002867D1CFE0C00639
:10B23000984AC00E012860D19449487800285CD013
:10B2400010798978884258D294494118944801600D
:10B25000FFF750FDBBE00027C006C00E3E46039737
:10B260000197012849D189484178002945D000211A
:10B2700002918C490978002902D1C17801293CD07A
:10B28000C17800290BD0884C2178002965D06078DE
:10B29000022806D004280ED0052859D11DE0834C81
:10B2A000F2E77A4861794078814251D0E078A1781C
:10B2B000000208434DE0A778E67800200190754829
:10B2C0000179B94244D18078B04241D10120029045
:10B2D0007248C15D0391C6553AE06E490879B8429B
:10B2E00036D1A0788F22104000900006009806D535
:10B2F0000007000F01252D0402E059E039E0012587
:10B3000085408878B04213D16048816829438160C4
:10B31000C168A943C1602046FFF7C0FC0098FFF751
:10B320001DFD009801F0D8FE0198284301900FE020
:10B33000039886420CD10198284209D1534881686C
:10B34000A9438160C168A943C1600098FFF7F2FC7E
:10B35000207804192078002899D10298002827D055
:10B3600000221146802001F031FF5148006800287A
:10B370002DD080472BE0C006C00E19D0012817D170
:10B3800000F048F9002822D100F0B0F900281ED1C1
:10B3900000F0E4F800281AD10AE0C006C00E07D178
:10B3A00000F0DEF9002812D100F028FA00280ED1B2
:10B3B00038480178C90904D1C088002801D000208C
:10B3C00000E0802001F0E4FE3549002088800498E8
:10B3D000400709D52F4D2878C00915D03548364982
:10B3E0000278002001F0E4FC0498000740D52948C9
:10B3F0000078C00932D02A48244980880979084356
:10B4000036D0FFF777FC33E0254CA288002AEBD03A
:10B410000020216801F0CCFC216809182160A18876
:10B42000081A0004000CA080DED128784106890F9C
:10B430000ED001290CD1C006C00E09D0012807D1B9
:10B4400000F06EF80028CFD100F038F80028CBD1FA
:10B45000802001F09DFE0020A080C5E70B49087800
:10B46000020605D54006400E0870002101F086FE58
:10B470000498400602D50020FFF702FC049800065D
:10B4800002D58020FFF7FCFB05B0F0BD8CF2FF1F5A
:10B4900001000100A8F2FF1FD03E010097F1FF1F3D
:10B4A000A0F2FF1F4B3E010085400100F93F010063
:10B4B000D43E0100503E0100301B002010B515495C
:10B4C000154A08791278904203D0144A12789042B3
:10B4D0001DD14878002804D0022807D0202816D192
:10B4E0000DE0FFF79FFB00280DD110E0C8788978A8
:10B4F00000020843FFF798FB002804D107E0FFF79C
:10B500009DFB002803D001F059FE012010BD002052
:10B5100010BD0000A8F2FF1F6E3E01006F3E01004B
:10B5200010B50B490B4A08791278904203D00A4AA9
:10B53000127890420AD14878092807D100F0A0FB80
:10B54000002803D001F03AFE012010BD002010BDFC
:10B55000A8F2FF1F513E0100523E010070B528497C
:10B56000284A08791278904203D0274A12789042EC
:10B5700043D123484978C27883781002234C244D64
:10B580001843042923D008DC002916D001290DD046
:10B59000022912D0032930D111E020290DD0212910
:10B5A0001AD022291DD0232927D11FE0FFF724FA22
:10B5B000002808D121E0012070BD2C60FBE7FFF7D7
:10B5C00019FA002819D02C60FFF794FBF3E7FFF776
:10B5D00001F900280ED110E0FFF710FA0028F2D18F
:10B5E0000BE0FFF723FB002804D106E0FFF7F2FA97
:10B5F000002802D001F0E2FDDDE7002070BD000070
:10B60000A8F2FF1F6E3E01006F3E0100301B0020BC
:10B61000A0F2FF1F10B52D4C2D49207909788842E2
:10B6200003D02C49097888424DD160780C284AD241
:10B6300001007944097949188F4445052834454566
:10B640004545451A2D3E00F033FA00283BD0E078FE
:10B65000012802D0032804D006E020491E480860D3
:10B6600002E01E491E480860FFF744FB012010BDA0
:10B67000E078022802D0032804D011E017491948C5
:10B6800008600DE015491648086009E000F0F8F977
:10B6900000280BD117E000F0CBFA002810D112E0FF
:10B6A000012010BD00F0FAF900280CD00B490E481B
:10B6B0000860FFF71FFBF3E700F0D8FA002802D07C
:10B6C00001F07CFDECE7002010BD0000A8F2FF1F98
:10B6D000513E0100523E0100711B0020A0F2FF1FED
:10B6E000A2F1FF1FB21B0020301B002010B518482C
:10B6F000184A01791278914227D142780146C878D8
:10B700008B7800021843CB798C7919022143FE2AE9
:10B710000CD0FF2A19D1002817D1002915D101F02A
:10B720007FFA002811D001F049FD0CE000280CD16F
:10B7300001290AD100F0EAFE002806D00749064890
:10B740000860FFF7D7FA012010BD002010BD0000EF
:10B75000A8F2FF1F643E0100301B0020A0F2FF1F73
:10B76000F8B5204D2049687809780027884236D1FD
:10B770006879297900020843022830D1AA781B4C45
:10B78000002A2CD000200126012A07D9217800297F
:10B7900000D00C19811C401C8A42F7D82078002860
:10B7A00018D003F057FA0146E01CFCF7CFFF104A0F
:10B7B00001271460E979AB792078090219438142A5
:10B7C0000AD90C4990800978491E084205D10A48D7
:10B7D000067002E0002702E09180FFF78BFA3846FE
:10B7E000F8BD0000A8F2FF1F7A3E010058F1FF1FCC
:10B7F000A0F2FF1F503E010090F2FF1F10B5154A46
:10B800001549507809780024884220D1507911795F
:10B810000002084307281AD1114B10481860417ADA
:10B82000007A09020143D079927900020124104381
:10B83000884209D90B4899800078401E014204D102
:10B8400009490120087000E09880FFF753FA20466C
:10B8500010BD0000A8F2FF1F7B3E0100163F010053
:10B86000A0F2FF1F503E010090F2FF1F0748002189
:10B870004170C16001614161418081808161C1612C
:10B88000C18001810162418170470000B0F2FF1F59
:10B89000F8B5494EB0887188484F00257C1C884215
:10B8A00018D3B069002815D17561B58001233978A6
:10B8B0007A1C184606F066FD70807088002809D052
:10B8C0003F4877610078012801D8746102E07088F0
:10B8D000401C7080708800283AD1F068002801D0A0
:10B8E000F56035E03069002832D035490978012902
:10B8F0000ED83D70B58002237A1C0021012006F08D
:10B9000041FD70807088002800D0746135611FE0AF
:10B910003C780127202C00D300243946A140014265
:10B920001AD0601CC1B2254A02231170B5800120D3
:10B93000521C06F027FD70807088002804D01F4834
:10B9400070617088401C70803069A740B8433061D6
:10B950007088002806D102E0641CE4B2DAE7B0691E
:10B96000002826D07088B188164F401A84B23878E3
:10B9700041001548405AA04200D204461348802195
:10B98000007822460843716901F020FC7069104973
:10B9900000197061B088001980B2B08009888842AF
:10B9A00008D2387841000848405AA04202D101200C
:10B9B000B061F8BDB561F8BDB0F2FF1F701B00208B
:10B9C0005E3E01008FF2FF1F5A3E0100533E010010
:10B9D000603E0100F8B51C4C002620891B4D1C4F11
:10B9E000002803D1E5613888E0802681E08821893C
:10B9F000421A1848E169007801F0DAF9E16980B289
:10BA00000918E161218909188BB22381002809D026
:10BA100039888B4206D21049104A09784900515A98
:10BA2000814210D90E48017801200129009003D8E5
:10BA30000021064A022003E029786A1C02205B1ECE
:10BA400006F02CFD2681F8BDB0F2FF1FB11B0020CF
:10BA5000623E0100543E01008FF2FF1F5A3E01007A
:10BA60005F3E010010B50446000702D52046FFF7EF
:10BA70000FFF600702D52046FFF7ACFF10BD0000A6
:10BA8000034804498078085C034908700120704726
:10BA9000A8F2FF1FA0F1FF1F301B002010B506F019
:10BAA0006FFC02490870012010BD0000301B00200F
:10BAB0000B490022C878012806D0022806D00328A6
:10BAC00006D1084A521C03E0074AFBE700207047F2
:10BAD00010B58978002306F055FC012010BD000048
:10BAE000A8F2FF1FA1F1FF1F701B0020474800783C
:10BAF00000287DD0F8B546480423017800264A1C6A
:10BB00000270444800784200821893405B1E9942BC
:10BB100003DB00233E4901260B703F4B00251988AB
:10BB2000FF2901D2491C198041003C48405A3A493A
:10BB300000900988884200D1012539490020097800
:10BB40008E4600294FD9022191408C460022002EBA
:10BB50000DD034490B5CFF2B01D25B1C0B54324BD4
:10BB60001B5C002B03D0095C994200D301222E49B3
:10BB70006446095C0B46A340009CA34203DA0029FB
:10BB800001D0012300E00023002D08D0002B06D0B7
:10BB90001F4F01243F6984403C431D4F3C61234CAF
:10BBA000245CA1420ED01F49095CA14208D3184F62
:10BBB00001213F6981403943154F396100213970B6
:10BBC00019490C54002A0AD0002B05D11049012232
:10BBD0000B6982401A430A61124900220A54401C30
:10BBE000C0B27045B2D3002D04D000210A4800E055
:10BBF0000AE0018006480169002904D04088002835
:10BC000001D1FFF745FEF8BD704700008DF2FF1F20
:10BC1000B0F2FF1F8FF2FF1F9CF1FF1F563E010085
:10BC20005E3E01009EF1FF1F9FF1FF1FA0F1FF1F6D
:10BC30000A480A498078C978002802D0084A815405
:10BC40000AE0084A00201378002B05D9064A11544F
:10BC5000401CC0B29842FAD301207047A8F2FF1FDF
:10BC60009FF1FF1F5E3E0100A0F1FF1F10B50348CA
:10BC7000807806F011FC012010BD0000A8F2FF1F23
:10BC80000D490022C878012806D0022806D00328D2
:10BC900006D10A4A521C03E000207047084AF9E71F
:10BCA00038B500230093CB798C791B022343897824
:10BCB00006F0F4FB012038BDA8F2FF1FA1F1FF1F21
:10BCC000B11B0020F8B5EFF31080C007C00F72B6AB
:10BCD000624D0026EC68EE60297800912E700028F5
:10BCE00000D162B6E00708D001F0AEF906F0C2FC60
:10BCF0005B480068002800D08047E00609D5594815
:10BD0000017920221143017157480068002800D0B2
:10BD10008047A00609D553490879DF2210400871F1
:10BD200052480068002800D08047600704D550487A
:10BD30000068002800D08047022C09D14D480168D6
:10BD4000002902D04748007A88474648FF210172FF
:10BD5000200779D5EFF31080C107C90F72B6AA6822
:10BD60006868904201D1012000E00020002900D144
:10BD700062B6002868D1404FEFF31080C607F60F77
:10BD800072B63E4968680C5C1521401CFCF79FFDAB
:10BD90006960002E00D162B620462207D30F21062B
:10BDA0006207090FD20F002908D15C00A418E40033
:10BDB0003C5D0026A406240F0D2C0AD08C005B00ED
:10BDC000E3189A18D600BA5D9206120F012A13D012
:10BDD0001DE02969022081432961387E4006400E1A
:10BDE0003876387C4006400E387425486E700168FD
:10BDF000002917D0022014E0002902D1C007C00F8B
:10BE000068701F480159002901D004208847B85D97
:10BE10008006000F092805D119480159002901D0D1
:10BE200008208847EFF31080C107C90F72B6AA68CF
:10BE30006868904202D1012001E005E0002000295D
:10BE400000D162B6002897D00098002804D0054899
:10BE5000017DDF2211400175F8BD0000A4F1FF1F34
:10BE60007C3E010080200740803E0100843E0100AE
:10BE7000883E01008C3E0100001E0020A02300200F
:10BE8000903E010010B41C48402303701B484168D9
:10BE90000522120411434160416B1A0311434163AF
:10BEA0001749900108601748017B802211430173F4
:10BEB000017B0906FCD41449144C090A2177124964
:10BEC000134A090C11741049090E1175FF212170D4
:10BED00010490968002900D004210F4A1268002A7D
:10BEE00000D0022211431922114321710370017BFA
:10BEF0001943017310BC7047B8F1FF1F0080044064
:10BF000000E100E000210740001E002080200740E3
:10BF1000A0200740883E01008C3E010070B500F073
:10BF200027F9002845D02348022202704270224D92
:10BF300003202A632870214C082021180B7818460A
:10BF40004B781B0218438B78C9781B0418430906E9
:10BF5000084302280ED91A48110A02724172110CC4
:10BF60008172110EC1722272100A6072100CA072DE
:10BF7000100EE07213488021007808430D4901F04B
:10BF800025F9082021180A7810464A781202104331
:10BF90008A78C9781204104309060843296B401AAD
:10BFA0002072010A6172010CA172000EE072012080
:10BFB000207370BDF21B0020D4F2FF1FDF2500208C
:10BFC000C0250020653E010010B51C4A11780029EB
:10BFD0000FD0012910D01A48052900781AD0072956
:10BFE00026D000F099FE17490220087300F076FE73
:10BFF00010BD00F065F910BD1348C07B2A2803D09E
:10C000002F2804D0AA28F6D100F0B6FB10BD00F00E
:10C0100033FB10BD012181400C480068014201D072
:10C02000012000E000200A4A0AA101F05BF910BDDE
:10C0300000201070106B1F28DBD010BDD4F2FF1F42
:10C04000663E0100DF250020C025002098F2FF1F7A
:10C050004A0400002E2E5C2E2E5C2E2E5C736F7513
:10C060007263655C7573625C6D73635C7573626447
:10C070005F6D73632E63000070B51C4B5868D86009
:10C08000002801D0012070BD194D082029180A7818
:10C09000184C10464A78120210438A78C978120464
:10C0A0001043090608431BD0287B000604D512481C
:10C0B00080210078084311E0082021180A781046F2
:10C0C0004A78120210438A78C9781204104309068C
:10C0D0000843196B884203D00848007800F01CFE22
:10C0E0000120207300F0FAFD002070BDD4F2FF1F84
:10C0F000C0250020DF250020653E0100663E0100CE
:10C1000010B5164801798F200140080605D50807AB
:10C11000000F01221204824001E001228A401048EF
:10C12000802300781843884216D10E4909681142CD
:10C1300012D00D4A1378194653781B02194393788D
:10C14000D2781B04194312061143084A914203D1C5
:10C150000D22054901F03AF810BD0000A8F2FF1FBA
:10C16000653E010098F2FF1FDF2500205553425322
:10C1700070B5104B082019180A78022410464A7826
:10C180000D4D120210438A78C97812041043090633
:10C190000843002806D0187B000608D4074800781A
:10C1A00000F0BAFD2C7300F099FD002070BD012055
:10C1B00070BD0000C0250020DF250020663E010084
:10C1C00010B51B491B4C0A7810464A7812021043DE
:10C1D0008A78C9781204104309060843216B884203
:10C1E00002D82063032000E0042020701248802140
:10C1F0000078226B0843114900F0E8FF104908203D
:10C200000A181378184653781B0218439378D2788B
:10C210001B04184312061043226B801A0872020A8C
:10C220004A72020C8A72000EC8720020087310BD98
:10C23000C8250020D4F2FF1F653E0100F21B00203C
:10C24000DF25002070B50446174D400709D5174873
:10C25000174902881748007800F0AAFD2863FFF705
:10C26000B3FE20070AD52878022808D003280FD06B
:10C27000042810D0052801D10020287070BD0E4878
:10C28000C07B282801D0A828F8D100F077F970BD2C
:10C2900000F024FD70BD094880210078084300F0BB
:10C2A0003BFD00F01BFD70BDD4F2FF1F6C3E010092
:10C2B000F21B0020663E0100C0250020653E010003
:10C2C000F8B58A4E326B1F2A01D2114600E01F21B9
:10C2D0000020874F002905D9864B1C5C3C54401C2C
:10C2E0008842FAD3844880210078012508431F2A18
:10C2F0006FD13B78FA7819467B7812061B021943F6
:10C30000BB781B04194311437C4A914261D13B79AC
:10C31000FA7919467B7912061B021943BB79784CCE
:10C320001B041943114321710A0A62710A0CA2719C
:10C33000090EE17108217A181378194653781B0207
:10C3400019439378D2781B041943120611432172C2
:10C350000A0A62720A0CA272090EE172797B012943
:10C3600004D8B97B002901D0102901D9257383E0B5
:10C37000F97B2A293BD021DC1A294ED00EDC042976
:10C38000F4D006DC00293BD00329EFD100F004FCF7
:10C39000F8BD1229EAD100F0C5F8F8BD232942D032
:10C3A00007DC1B292FD01E29E0D1F87CC007DDD186
:10C3B0007EE025293AD02829D8D140E09E293BD0DB
:10C3C0000DDC5529D2D005DC2F2958D03529CDD107
:10C3D00058E072E05A2923D09129C7D152E0A1290F
:10C3E00027D0A32966D0A82929D0AA29BED100F038
:10C3F000E3FA0028D1D0387B000635D43570F8BD7B
:10C4000000F0A0FCF8BDB87C0028AFD1F87CC007D4
:10C41000C00F706006F0F4F834E000F08DFAF8BD5B
:10C4200000F048FAF8BD00F069FBF8BD00F040FBF1
:10C43000F8BDFFF773FDF8BD00F018FCF8BD00F083
:10C44000BBFA0028FAD0387B000604D502203070F1
:10C4500000F094F8F8BD2B48007800F05DFC022055
:10C46000207300F03BFCF8BD23488021007808438E
:10C4700000F052FC0220207300F030FCF8BD387C44
:10C48000800704D40020207300F028FCF8BD00F0E1
:10C4900093FA0028FAD0387B000602D43570356252
:10C4A000F8BD154880210078084300F035FC0220D3
:10C4B0002073E1E700F030FC58E70F4C00F02CFC53
:10C4C0002078114C0107090F0120000488402168E1
:10C4D0000C4F08432060387800F01EFC3878854007
:10C4E00020680543062025603070F8BDD4F2FF1F98
:10C4F000C0250020F21B0020653E01005553424339
:10C50000DF250020663E01009CF2FF1F10B506F0FB
:10C5100099FD0349002800D001200870012010BDBA
:10C52000301B002010B5FFF723FE00281FD0104B52
:10C53000002018708021597002219970D970202430
:10C540001C7158719871D8710A48016808200A78DE
:10C55000002A02D01A54491C00E01C54401CC0B2EE
:10C560002428F4D3044924200863FFF729FE10BDD2
:10C57000F21B002054F1FF1FD4F2FF1FF8B5384D15
:10C580000026A969686A374F88420AD33648802155
:10C5900000780024084300F0BFFB3E7300F09EFBD0
:10C5A00008E03248007841003148445AE86A844241
:10C5B00000D30446FFF760FD002800D10024A86ADC
:10C5C000002839D0002C0FD0A96AE86980224118D0
:10C5D000254800781043224600F0F8FDA86A0019AB
:10C5E000A862E86A001BE86229696869AA6A41438F
:10C5F000914203D1AE62696A08186862082039184E
:10C600000A7810464A78120210438A78C9781204D0
:10C61000104309060843001B3872010A7972010CA5
:10C62000000EB972F872002C05D0E86A002802D119
:10C63000032028703E73F8BD002CD5D02969E86A24
:10C640004018401EFCF743F969690246884200D948
:10C650000A460848E969437B686A05F0B1FFB3E719
:10C66000D4F2FF1FDF250020653E01008FF2FF1F7F
:10C67000683E0100C0250020F8B53A4C0025A169AC
:10C68000606A884208D338482563007800F044FB8C
:10C690003648057300F022FBFFF7EEFC002806D0B9
:10C6A000206B002827D0A06A002802D012E0256362
:10C6B00021E02169E06A4018401EFCF708F9616931
:10C6C0000246884200D90A462948E169437B606AEC
:10C6D00005F076FF276B0020002F0CD9A66AE369CE
:10C6E00031185A5C2349095C8A4201D0256202E074
:10C6F000401CB842F4D3236BA06AC018A062E16A60
:10C70000CE1AE662226961694A43824203D1A56278
:10C71000606A40186062154908200A181578284692
:10C7200055782D0228439578D2782D042843120697
:10C730001043C01A0872020A4A72020C000E8A7272
:10C74000C872002B0BD0002E02D02078052806D10D
:10C75000206A002804D00020087300F0BFFAF8BD5A
:10C760000120F9E7D4F2FF1F663E0100DF2500201B
:10C77000C0250020F21B0020F8B5404D0024A96917
:10C78000686A884208D33E482C63007800F0C4FAF7
:10C790003C48047300F0A2FAFFF76EFC002800D1B9
:10C7A0002C63296BA86A2A694018904206D9FF2297
:10C7B0000A3235A1002000F095FDF8BD00200029C7
:10C7C00009D93A4EEB69AA6A315C12189954296B5F
:10C7D000401C8842F7D3A86A4018A862EA6A521A35
:10C7E000EA62002927D0324F002A15D1002813D041
:10C7F00029694018401EFCF76AF8696906468842B4
:10C8000000D90E467B7B3246E969686A05F0FAFE7C
:10C81000AC62686A80190DE06A69296951438142F6
:10C8200009D17B7BE969686A05F0ECFEAC62696955
:10C83000686A40186862134908200A181378184675
:10C8400053781B0218439378D2781B0418431206BE
:10C8500010432A6B801A0872030A4B72030C000EF5
:10C860008B72C872002AA8D0E86A002802D0287803
:10C870000528A2D10C7300F031FAF8BDD4F2FF1FE5
:10C88000663E0100DF2500202E2E5C2E2E5C2E2E13
:10C890005C736F757263655C7573625C6D73635C0A
:10C8A000757362645F6D73632E630000F21B00207A
:10C8B000C025002010B5FFF75BFC002833D0FFF740
:10C8C000DBFB00282FD0184800210170062242709F
:10C8D000164B81701A7AD201C27001714171817157
:10C8E000C1710821124A196353181C7820465C78DC
:10C8F000240220439C78DB78240420431B06184341
:10C9000008280ED90B480B0A017243720B0C837274
:10C910000B0EC3721172080A5072080C9072080E46
:10C92000D072FFF74DFC10BDF21B0020D4F2FF1FA8
:10C93000DF250020C025002010B5FFF719FC0028D6
:10C9400030D0FFF799FB00282CD017480321017045
:10C950000021164B41701A7AD2018270C1700421F5
:10C96000134A0820196313181C7820465C782402A7
:10C9700020439C78DB78240420431B0618430428BA
:10C980000ED90C480B0A017243720B0C83720B0E0A
:10C99000C3721172080A5072080C9072080ED0729D
:10C9A000FFF70EFC10BD0000F21B0020D4F2FF1FA9
:10C9B000DF250020C025002070B5374D1020291834
:10C9C0000A78364C10464A78354E120210438A785F
:10C9D000C978120410430906084300BA010A207DF1
:10C9E0000902014300207162B062E07B2F280AD067
:10C9F00004DC28280BD02A2825D104E0A82810D050
:10CA0000AA2820D109E0FFF737FB002841D0E07DBC
:10CA1000A17D0002084341BA15E0FFF72DFB002875
:10CA200037D0142029180A7810464A781202104389
:10CA30008A78C978120410430906084300BA010A2B
:10CA4000207E090201433069012541430820221854
:10CA5000F1621378134E184653781B0218439378EB
:10CA6000D2781B0418431206104300280DD08842C8
:10CA700010D0207B000604D50B48802100780843A5
:10CA800001E00A48007800F047F9357300F026F914
:10CA9000002070BD012070BDC1250020C0250020F0
:10CAA000D4F2FF1FDF250020653E0100663E010035
:10CAB00010B5FFF75DFB00281AD0FFF7DDFA00285C
:10CAC00016D00C4A0C499069401E030E0B70030CE3
:10CAD0004B70030A8B70C8701069030E0B71030C46
:10CAE0004B71030A8B71C87108201063FFF768FB54
:10CAF00010BD0000D4F2FF1FF21B002010B5FFF79D
:10CB000037FB00283ED0FFF7B7FA00283AD01E487E
:10CB1000002101704170817008211C4AC170916927
:10CB20000B0E03710B0C43710B0A8371C17102214F
:10CB3000017211690B0C43720B0A8372C1720C21D2
:10CB40001163134A082013181C7820465C782402CD
:10CB500020439C78DB78240420431B0618430C28D0
:10CB60000ED90C480B0A017243720B0C83720B0E28
:10CB7000C3721172080A5072080C9072080ED072BB
:10CB8000FFF71EFB10BD0000F21B0020D4F2FF1FB8
:10CB9000DF250020C025002070B5FFF7E9FA002846
:10CBA0002ED01C487021017000211B4B41705A6827
:10CBB000DD681446AC4306D0062484702824047330
:10CBC0004173DA600AE0002A1BD0144A127B002A63
:10CBD0001DD005228270202202734173C170017141
:10CBE000417181710A22C271017241728172C172F6
:10CBF0008173C1730174417412201863FFF7E0FA66
:10CC000070BD022282703A2202734173E6E781709E
:10CC10000173E2E7F21B0020D4F2FF1FDF250020A2
:10CC20000649002008600649087048708870C8707E
:10CC30000449072008700120704700009CF2FF1F84
:10CC4000DF250020D4F2FF1F0549002008600549B8
:10CC5000087048708870C8700349072008707047D2
:10CC60009CF2FF1FDF250020D4F2FF1F10B5FFF755
:10CC70007FFA002829D01548202202700021417037
:10CC8000C177134C03202263207012488021007862
:10CC900008430E4900F09AFA0F4908200A18137841
:10CCA000184653781B0218439378D2781B04184314
:10CCB00012061043226B801A0872020A4A72020C92
:10CCC0008A72000EC8720120087310BDF21B00208A
:10CCD000D4F2FF1F653E0100DF25002010B50A4891
:10CCE0000A49020A08704A70020C8A70000EC87065
:10CCF0000748802100780D220843044900F066FAB5
:10CD000004490520087010BD55534253DF2500200B
:10CD1000653E0100D4F2FF1F10B5044600F038FA5A
:10CD2000200605D52107090F01200004884001E0F5
:10CD30000120A04002490A681043086010BD0000AD
:10CD400098F2FF1F154B10B5082019180A78144CDB
:10CD500010464A78120210438A78C97812041043A8
:10CD60000906084310D0187B000604D50D48802121
:10CD70000078084301E00C480078FFF7CDFF012060
:10CD80002073FFF7ABFF10BDFFF776F90028FAD04C
:10CD900000202073FFF7A2FF10BD0000C025002077
:10CDA000DF250020653E0100663E0100704700005F
:10CDB000F7B5064682B0002000903007850E3D484A
:10CDC000EC0020180F4601904188002E1DD13A48F2
:10CDD0004078002811D0680801218140EFF31080CD
:10CDE000C007C00F72B6354A13684B401360002865
:10CDF00000D162B6002005B0F0BD2E48005D80066F
:10CE0000000F0D2801D1012000900498884206D21D
:10CE1000FF22EF322AA1002000F064FA04990020DA
:10CE2000002907D9334BAA01D3181A5C3A54401C85
:10CE30008842FAD33048825D01981E4E42801E48D7
:10CE40006A080069355D0346D340DB076D06DB0FDA
:10CE5000ED0FAB4214D1FB79BD791B022B43009D32
:10CE6000002D01D0002B12D001259540EFF3108347
:10CE7000DB07DB0F72B6114F68403860002B11D012
:10CE80000D480069D040C0070ED0C8200DE0EFF378
:10CE90001083DB07DB0F72B6084D400840002860A6
:10CEA000002BEDD162B6EBE788203055084605B07F
:10CEB000F0BD0000001E0020A4F1FF1FB4F1FF1F11
:10CEC0002E2E5C2E2E5C2E2E5C736F757263655C4D
:10CED0006869635F68616C5C667265657363616CE9
:10CEE000655C757362645F6B696E657469732E63EC
:10CEF00000000000A01E0020B8F1FF1F10B5FFF7D2
:10CF0000FFF810BD70B41B4A1B4CD3781B4A257820
:10CF10001478184A1A4E1279212B02D0222B25D1CF
:10CF200018E0AA4201D0A24220D1164A1378164A2C
:10CF3000002B127801D1012A18D0002A08D0134AF8
:10CF400002601046124A128880183060092009E0F9
:10CF5000104AF5E7AA4201D0A24207D10E4830603C
:10CF60000E480088086070BC0120704770BC00202B
:10CF700070470000A8F2FF1F513E0100523E010021
:10CF8000A0F2FF1F4B3E01008FF2FF1F8540010002
:10CF9000003F0100F93F0100DC3E0100FE3E0100C0
:10CFA00070B5274B024618782549C0064988254E9A
:10CFB000C00E04D001282BD0022829D111E001296C
:10CFC00026D10224002A05D0012000F0FEF8F088C6
:10CFD000204304E0002000F0F8F8F088A043F0803F
:10CFE0002CE01D798F200540280605D52807000F65
:10CFF00001242404844001E00124AC40707800281E
:10D0000006D0280704D0B068204201D0002901D002
:10D01000002070BD002A05D0284600F0B9F8F0685D
:10D0200020430AE03069204208D12846FDF728FE57
:10D030002846FFF763FFF068A043F060012070BD51
:10D04000A8F2FF1F8CF2FF1F70B5012618483606A4
:10D0500006600120174D0024810049190C70401C06
:10D060001028F9D315211448FBF72FFC1348144955
:10D0700044608460C4600470447040224A80114A55
:10D080004A60C8220A700C720F4ACC614A610D21B5
:10D0900029700E4901610E48017D0222114301757C
:10D0A000FF2101700172017304760A48066070BDA9
:10D0B00080E100E0C0200740A0230020A4F1FF1F72
:10D0C000001E0020A01E0020201F00205555555591
:10D0D0008020074000E100E0F0B41E4F0107040685
:10D0E000002601231C4D090F3A68002C16DA48006F
:10D0F000401C8340EFF31080C007C00F72B61A4384
:10D100003A60002800D162B60A0214481218480199
:10D1100040198032C6614261F0BC70474400A340B0
:10D12000DC43EFF31083DB07DB0F72B622403A607B
:10D13000002B00D162B60A4A135C4A0150194380A1
:10D140000B020649591841608821A9540672F0BCA7
:10D1500070470000B4F1FF1F001E0020A01E002039
:10D16000B8F1FF1F10B5FDF7F1FCFFF76DFD10BD25
:10D1700010B5FEF7BBFCFDF7EDFC10BD002903D197
:10D1800040060249400E08767047000080200740A4
:10D190000007810E0348081801780222114301702C
:10D1A00070470000C020074010B503488168012087
:10D1B000400201F0BFFE10BD60F0FF1F10B500225D
:10D1C0001146802000F002F810BD7047F0B400074F
:10D1D000800E801C144FC600F3195A800023002AC9
:10D1E00007D9124D84016419CD5CE5545B1C934250
:10D1F000FAD341080E4800690346CB40DB0701D053
:10D20000882300E0C823BB5501238B40EFF3108136
:10D21000C907C90F72B6074C58402060002900D1D9
:10D2200062B61046F0BC7047001E0020A01E002011
:10D23000A4F1FF1FB4F1FF1F00207047002101601F
:10D240004160017270470A7802704B7843708A78A7
:10D250008270CA78C2700B790371704710B4002ACB
:10D2600006DA52005208D21DD308DB00102203E078
:10D27000D21C93089B000C22002B02D09C188C42DD
:10D2800002D910BC012070478218836041180260E7
:10D290004160C91AD018884202D810600246F9E7E6
:10D2A0000020106010BC7047B0B5044603F07EFA51
:10D2B000002804D0034F0249BC46206800DFB0BDFF
:10D2C000FFFF000029020100B0B5044603F06EFA2A
:10D2D000002803D0024F2068BC4600DFB0BD00002C
:10D2E0007D01010000281FD1F8B516460F46EFF367
:10D2F0001080C407E40F72B600231A461946184678
:10D3000000F098FA050003D13146384600F0E6FAFD
:10D31000002C00D162B6002D05D1EFF30380C006CA
:10D3200001D105F09BFDF8BD7047704770B51149FC
:10D330000F483CC93CC03CC93CC04A6809684260CF
:10D34000016005F04FFF0C4805F040FF05F04AFC76
:10D350000A49012208600A4952020A60094A012169
:10D3600011600949400A086009490848086070BD11
:10D3700044060020383A010051E0000008F3FF1F86
:10D38000E4F2FF1FE8F2FF1FECF2FF1F440400204D
:10D39000F0F2FF1F10B590B04021684604F006FD82
:10D3A00004000AD06846007803F0AEFA21466846C9
:10D3B000FDF72EFA012001F0EBFD40216846FDF754
:10D3C0000BFA002806D081B2684604F05DFD01200A
:10D3D00001F0DEFD01F0F4FD10B010BD10B4EFF36C
:10D3E0001081CB07DB0F72B6EFF31081CC07E40F8F
:10D3F00072B64268016880688A4201D3511A01E01E
:10D400001218511A002C00D162B6401A401E002B8F
:10D4100000D162B610BC7047EFF31081CB07DB0F71
:10D4200072B6426801688A4201D3501A02E08068ED
:10D430001018401A002B00D162B67047EFF310832A
:10D44000DB07DB0F72B68260C160002101604160C2
:10D45000002B00D162B6704770B50446EFF3108020
:10D46000C507ED0F72B661682068884201D00120BF
:10D4700000E0002043220D49FFF734FFE1682068F7
:10D480000E5C401C2060A16888420AD3884201D10A
:10D49000012000E0002048220449FFF723FF00207C
:10D4A0002060002D00D162B6304670BD04D500006A
:10D4B00070B50446EFF31080C507ED0F72B66268D1
:10D4C000E06881546068401C6060A16888420AD3AB
:10D4D000884201D1012000E00020312209A1FFF79C
:10D4E00001FF0020606061682068884201D001204F
:10D4F00000E00020362203A1FFF7F4FE002D00D14A
:10D5000062B670BD2E2E5C2E2E5C2E2E5C736F7557
:10D510007263655C6461706C696E6B5C6369726395
:10D520005F6275662E630000F7B582B00446EFF3C4
:10D530001080C307DB0F72B661682068814201D397
:10D540000E1A02E0A56849190E1A002B00D162B626
:10D55000B24200D216460025002E2CD9EFF31080DF
:10D56000C707FF0F72B661682068884201D00120AA
:10D5700000E0002043221149FFF7B4FEE168206873
:10D58000095C401C00912060A16888420AD388424F
:10D5900001D1012000E0002048220849FFF7A2FE47
:10D5A00000202060002F00D162B6039900984855F2
:10D5B0006D1CB542D2D3304605B0F0BD04D5000095
:10D5C000F7B50446EFF31080C607F60F72B6EFF317
:10D5D0001080C507ED0F72B663682168A0688B42A2
:10D5E00001D3591A01E01B18591A002D00D162B657
:10D5F000401A401E002E00D162B6824200D2104670
:10D600000025064600282BD90198405DEFF31081D4
:10D61000CF07FF0F72B66268E16888546068401CEB
:10D620006060A16888420AD3884201D1012000E0ED
:10D63000002031220C49FFF755FE00206060616830
:10D640002068884201D0012000E0002036220649EF
:10D65000FFF748FE002F00D162B66D1CB542D3D350
:10D66000304603B0F0BD000004D5000010B50B48F3
:10D67000C0780121C00948402A2209A1FFF732FEE3
:10D6800001246402224612491248FFF7D7FE2246BF
:10D6900011491248FFF7D2FE10BD000000B006404D
:10D6A0002E2E5C2E2E5C2E2E5C736F757263655C65
:10D6B0006869635F68616C5C667265657363616C01
:10D6C000655C6B6C32367A5C756172742E63000037
:10D6D00020170020101700203019002020190020EA
:10D6E00010B500F075FE10BD10B500F071FE10BD54
:10D6F00002488079002800D001207047A42500202E
:10D700000248C079002800D001207047A4250020DD
:10D710000248007A002800D001207047A42500208C
:10D72000F8B58C212648FBF7CEF8264E264F3278E6
:10D73000F17810467278090612021043B2788C25EF
:10D74000120410430843214CB84211D17079317949
:10D7500005020D438C2D01D22A4600E08C228C2D2F
:10D7600000D88C2517491648FAF7FCFF0020E07115
:10D770008C211448FBF7A7F83770390A7170390CFF
:10D78000B170390EF1703571290A71714122104959
:10D79000F01DFAF7E7FF607A227A01020D48114383
:10D7A0000172090A4172A17A8172E17AC1728A001A
:10D7B00009490A48FAF7D6FF00F0C8F8F8BD00009A
:10D7C00018250020002F0020646C766B582500205F
:10D7D0001F250020402F0020642500204C2F002012
:10D7E0000A4AD17A102901D300207047084B8900DA
:10D7F000C91840310873030A4B73030C8B73000E76
:10D80000C873D07A401CC0B2D0727047402F00203D
:10D81000002F002010B541210448FBF754F80448BC
:10D82000002101724172C17210BD0000072F00205B
:10D83000402F0020FFB581B01C4615460F46194801
:10D84000FAF7BAFD461C0198002802D03946FBF7CA
:10D850003AF80020002D00D02880002C00D0207045
:10D860001149C87900281AD0BE4201D8324602E0D8
:10D87000F01B41183A460198C91D0C4E002804D0EF
:10D88000707A337A000218432880002D02D0019864
:10D89000FAF768FF002C01D0B07A2070012005B0A3
:10D8A000F0BD0000072F0020002F0020402F002097
:10D8B0000449CA7A002A03D0034A0260C87A704732
:10D8C00000207047402F00204C2F00200248807914
:10D8D000002800D001207047002F0020F3B581B050
:10D8E0000546FAF769FD144E441C41273946F01DE0
:10D8F000FAF7E9FF412C02D82946224602E0413CD2
:10D9000061193A46F01DFAF72DFF0C4C029820726F
:10D91000000A607200F0EEF8002801D0012007E054
:10D9200000F0EAF8002803D00220A07203B0F0BD96
:10D93000A07203B0F0BD0000002F0020402F002097
:10D940000149887170470000002F002070B5002247
:10D9500011461046FCF7F8FA09221F491F48FAF74A
:10D9600001FF1F4C22781046627812021043A27801
:10D97000E1781204104309061A4D0843A8420FD15A
:10D980006079217900020843092804D2607921795D
:10D9900002020A4300E0092211491048FAF7E2FEA8
:10D9A0000E480921056081802278104662781202B3
:10D9B0001043A278E1781204104309060843A842F4
:10D9C00005D16079217900020843092802D2034871
:10D9D00001F044FE70BD00006A410100A425002052
:10D9E00000FC0100646C766B10B503498871084631
:10D9F00001F034FE10BD0000A425002010B503493D
:10DA0000C871084601F02AFE10BD0000A4250020C0
:10DA100010B503490872084601F020FE10BD000051
:10DA2000A4250020F8B586460020C04300268C4679
:10DA3000002921DD714608258B5D00242246D90787
:10DA400004D0A91A0127491E8F403C43521C5B0891
:10DA5000D2B2AA42F3D3210648400A4A082100283C
:10DA600002DA4000504000E04000491E0906090E5D
:10DA7000F5D1761C6645DDDB202102F047F9C04375
:10DA8000F8BD0000B71DC104F7B50C462021C04306
:10DA900002F03CF902990026A446002922DD6146E5
:10DAA00008258B5D00242246D90704D0A91A012736
:10DAB000491E8F403C43521C5B08D2B2AA42F3D3AA
:10DAC000210648400A4A0821002802DA4000504056
:10DAD00000E04000491E0906090EF5D10299761CA6
:10DAE0008E42DCDB202102F011F9C04303B0F0BD0F
:10DAF000B71DC104002070470120704710B50023F6
:10DB00001A4600F09FFC002800D0012010BD10B57F
:10DB100004F0B6FE012800D0002010BDF8B5164E66
:10DB20001F2530780024AD02012806D0FF223932AB
:10DB300012A10020FFF7D6FB0AE0B07802270028E8
:10DB400008D0FF223F320DA10020FFF7CBFB37703A
:10DB50000220F8BD204600F02DF8002802D03770D2
:10DB60001E20F8BD012080022418AC42F2D301200F
:10DB7000B0700020F8BD0000D4F0FF1F2E2E5C2EE8
:10DB80002E5C2E2E5C736F757263655C6461706CC5
:10DB9000696E6B5C647261672D6E2D64726F705C70
:10DBA0006961705F666C6173685F696E74662E632D
:10DBB00000000000F0B53B4E0446307883B00128E9
:10DBC00006D0FF22013238A10020FFF78BFB21E0B5
:10DBD0000127BF0239462046FAF779FE02250029BF
:10DBE00009D0FF22093230A10020FFF77BFB3570FE
:10DBF000022003B0F0BDF07800280ED0F168B068C4
:10DC00004018A04209D0FF22103227A10020FFF7C0
:10DC100069FB3570022003B0F0BD01227F20D203E2
:10DC200080020121944203D3844201D2002000E00B
:10DC30000846002831D0F1701F208002F760B460E0
:10DC4000844201D31F201CE0FFF756FF014622202B
:10DC5000002916D0002C14D10120C0030090C0115F
:10DC600000270190384600F0B9FD002801D00E20B1
:10DC700007E03846009A019900F02EFF002800D0F6
:10DC80001C20222804D00028C5D0357003B0F0BD78
:10DC9000204600F0A3FD0028F8D035701D2003B009
:10DCA000F0BD0000D4F0FF1F2E2E5C2E2E5C2E2E19
:10DCB0005C736F757263655C6461706C696E6B5CDC
:10DCC000647261672D6E2D64726F705C6961705F44
:10DCD000666C6173685F696E74662E630000000095
:10DCE000012080027047000010B5242804D20649A4
:10DCF00080000858002805D1E12204A10020FFF788
:10DD0000F1FA0AA010BD0000283901002E2E5C2E69
:10DD10002E5C2E2E5C736F757263655C6461706C33
:10DD2000696E6B5C6572726F722E6300000000009A
:10DD30000121242801D20249095C084670470000ED
:10DD40001CF0FF1FF0B50446054683B04018019053
:10DD500000E0641C2078402802D00028F9D15DE062
:10DD60006078622845D012DC522853D008DC422863
:10DD70003FD0442846D048283ED04D2817D132E025
:10DD800054283CD0552831D0562810D13EE0722876
:10DD900040D006DC642835D068282DD06D2806D107
:10DDA00021E074282BD0752820D076282ED01DA7EE
:10DDB0002046FAF701FB06463846FAF7FDFA0090CE
:10DDC00020188119019A891E914226D2B21EA11CE7
:10DDD000FAF72CFD39462046009AFAF7C3FC207862
:10DDE0000028B7D11AE000F09DFF0DE000F0A2FF7F
:10DDF0000AE000F02FFF07E000F068FF04E000F009
:10DE000095FF01E000F05EFF0746D1E700F09AFFC2
:10DE10000746CDE705480768CAE7A419601B03B0A9
:10DE2000F0BD00004552524F520000000C39010075
:10DE300030B58BB005F006F9002879D001225202E6
:10DE40003C493D48FAF744FA3B488021417400219F
:10DE500081740446207BE27A010211433748E41CB6
:10DE6000FAF735FDE51E697B354A4A43824203D8FD
:10DE7000344A4A43824200D2104601231B04002246
:10DE8000984205D32274120A62742B4A106204E08D
:10DE90002074030A6374284B1A62FAF718FD2A49A2
:10DEA00000024018040CEC82C0212848FAF70DFD4E
:10DEB0003C2227492548FAF70BFA244960024861B9
:10DEC000086224490520C86002220021684605F046
:10DED000C1F868460078204CF82803D1684640789D
:10DEE000FF2802D005F0DAF808E02022002102A87D
:10DEF00005F0ACF86846007AFF2819D105F0B9F8AA
:10DF0000164801466C312EC905950493039202917F
:10DF1000C06F06ADE369A26961690FC50B2210A14C
:10DF200002A8FAF7D5F92022002102A805F004F989
:10DF30000BB030BD803B0100BC0A002000B0FE00E9
:10DF40005A10000091FF000080FF00007C0F0020AD
:10DF5000B03D010010F1FF1FEC3D0100803D0100CC
:10DF6000464C41534820202020202000F7B582B0A5
:10DF70001546044605F066F800282AD000266902F6
:10DF80000398FAF7A0FC14490020CA68002A20D997
:10DF900031460C225143114A8B189B685B0AC31807
:10DFA000009384420CD39C420AD21F1BAF4200D381
:10DFB0002F465358201A3A4603999847E419ED1B07
:10DFC000002D06D00449761CC968F6B200988E422E
:10DFD000DED305B0F0BD000010F1FF1F7C0F002064
:10DFE000F7B582B01546044605F02CF8002826D077
:10DFF00014490026CA683046002A20D90C2132462E
:10E000004A43114952189168490A411800918442C3
:10E010000CD38C420AD20F1BAF4200D32F46536859
:10E02000201A3A4603999847E419ED1B002D06D0B3
:10E030000449761CC968F6B200988E42DED305B05A
:10E04000F0BD000010F1FF1F7C0F002070470000A2
:10E05000F8B51E4615460C46074605F08BF93149C2
:10E060000878032811D03048022C0FD0002C22D081
:10E07000012C0AD10268AA4207D18978002936D03A
:10E0800000214A1E016082608161F8BD0068A842DB
:10E09000FBD1304604F0F6FC0446304604F000FDA7
:10E0A0000646384602F066FE0346224631462846BA
:10E0B00003F01EFDF8BD384602F05CFE0328F9D0DF
:10E0C000304604F0DDFC8007F4D4384602F052FEFE
:10E0D0000746304604F0D6FC0446304604F0E0FC27
:10E0E00001463B462246284603F002FDF8BD0F4993
:10E0F000114F3CC93CC03CC93CC04A6809684260F9
:10E1000001600B490B48BC4600DF0C4881780129AF
:10E1100003D14178022900D18170094F0548BC46DE
:10E1200000DFF8BD6406002044060020383A0100F4
:10E13000FFFF00006C06002029020100F8F0FF1F1D
:10E140007D010100F7B50546444C0298A1784602CE
:10E1500000293AD13146019802F0F6FD032831D06A
:10E1600007466078002810D000203D4A3D49FFF75F
:10E17000B9F8681C00D001203B4A3A49FFF7B2F8D1
:10E180003A484168491C02D002E00120EDE74560B1
:10E19000E179032900D1E77134484168A94202D1ED
:10E1A000E079B84201D003200AE0384602F07CFD55
:10E1B000010004D12D4A0120D5606070A07008468E
:10E1C00003F0EAFCA078002811D0284F7868A84214
:10E1D0000DD8F868A8420CD0A84208D93869401C6C
:10E1E00000D13D613869A84200D205463D6103B0C7
:10E1F000F0BDF8698019F86102982818F860E07895
:10E20000002801D0002019E0019DF0051AD000205F
:10E21000174A1449FFF766F86078164A1149FFF764
:10E2200061F83146284602F0BFFD002510280BD0CA
:10E2300011280FD0257179698919796103F0ACFC37
:10E2400003B0F0BD0120E3E702F0ECFC65700121B2
:10E25000E17001E0002001212171ECE7640600205B
:10E260009E020000EC2F01009F02000044060020E7
:10E27000DD020000DE020000F0B585B019A10968DA
:10E2800004910378002104AA545C9C4227D0491CC5
:10E290000329F9D314A10A688E6896464A68CD68A6
:10E2A00000239446C25C7146009111466446613970
:10E2B000029603950194192911D9202A01D2052A21
:10E2C0000DD100216C46675C974208D0491C10298B
:10E2D000F9D35B1C0B2BE5D3012005B0F0BD00206A
:10E2E00005B0F0BDE5002000222A2B2C2E2F3A3B52
:10E2F0003C3D3E3F5B5C5D7C70B50446201E01D119
:10E30000042108E0C269002A04D01168022901D161
:10E31000002100E06D210D46002D00D070BD0449A4
:10E3200002480968884700BFF8E700000C3000F099
:10E330004CF1FF1F01680122920211430160BFF3FB
:10E340006F8FBFF34F8F70477047002801D10420B3
:10E35000704710B45B1E194201D11A4202D010BCA2
:10E360006520704703688B4204D8406889181818E4
:10E37000884202D210BC6620704710BC0020704753
:10E3800010B5114C70212170002811D0C0690028EF
:10E3900002D0006802280DD06D20002807D10B495B
:10E3A0002046096888472078810605D5672010BD7A
:10E3B0000420F2E70020F0E7C10601D5682010BD77
:10E3C000C007FCD0692010BD0000024048F1FF1FCB
:10E3D00070B50E4D00202C78002C0FD00021297034
:10E3E000A978002901D000F025FB022C05D069781E
:10E3F000032902D0002800D1212070BDFF22333232
:10E4000003A10020FEF76EFF022070BDA8F0FF1FE1
:10E410002E2E5C2E2E5C2E2E5C736F757263655CE7
:10E420006461706C696E6B5C647261672D6E2D64E3
:10E43000726F705C666C6173685F6465636F64655E
:10E44000722E630030B583B01C460546302901D3D7
:10E45000012000E00020402213A1FEF743FF2946DF
:10E460000C2220316846FAF77DF91C490198884250
:10E470000CD11B490098884202D1022003B030BD64
:10E48000184988420CD1012003B030BD284604F061
:10E4900085F9002801D1002C02D0032003B030BD43
:10E4A000002003B030BD00002E2E5C2E2E5C2E2EE0
:10E4B0005C736F757263655C6461706C696E6B5CD4
:10E4C000647261672D6E2D64726F705C666C61732F
:10E4D000685F6465636F6465722E63000199969747
:10E4E0008F9E939B939D939BFFB581B0064600241E
:10E4F00004982546002813D00A98002810D00499C3
:10E50000002008600A9907460860FFF7F3FA002820
:10E510001AD00120C003022E0AD0032E10D01BE017
:10E52000652225A10020FEF7DDFE022005B0F0BD2A
:10E530000399002904D00299814201D018240CE0EB
:10E5400007462A48056808E0FFF7D6FA002803D0F6
:10E55000012E07D0032E0FD01924FFF7D1F8002881
:10E560000FD010E00398002804D00298002801D0B2
:10E570001724F2E71D4802E01D4887681D4805681A
:10E58000EBE7012E04D0002C04D0204605B0F0BDEE
:10E590001924FAE7002D06D0049807600A98056050
:10E5A000204605B0F0BD9D2203A10020FEF79AFE93
:10E5B000022005B0F0BD00002E2E5C2E2E5C2E2E0B
:10E5C0005C736F757263655C6461706C696E6B5CC3
:10E5D000647261672D6E2D64726F705C666C61731E
:10E5E000685F6465636F6465722E6300343A01008E
:10E5F000E4F1FF1FFC39010010B50D4C2078002814
:10E6000006D0AC220BA10020FEF76CFE022010BD4C
:10E61000FF2230211448FAF731F901202070002040
:10E6200060706060A060E060A070E07010BD0000ED
:10E63000A8F0FF1F2E2E5C2E2E5C2E2E5C736F75A5
:10E640007263655C6461706C696E6B5C6472616757
:10E650002D6E2D64726F705C666C6173685F6465AB
:10E66000636F6465722E6300C8FBFF1FF7B54B4FE5
:10E670000546387884B01446012807D0C12248A145
:10E680000020FEF72FFE022007B0F0BDF87800282A
:10E6900003D1BD600120FD60F870B878002856D124
:10E6A000F9688D4201D1012000E000200919F960CC
:10E6B00000282FD0786830210E1AA64200D91646BD
:10E6C0004449324608180599FAF74CF87868A41BB3
:10E6D000801978600599AD1989190591302829D3D9
:10E6E00016D00020E3222EA1FEF7FCFD01233948BD
:10E6F000BA687968FFF7A6FE787001A8009002ABAF
:10E7000001227878B968FFF7EFFE002826D103E0F0
:10E710000120E7E70320EFE7B87801267040FC22EC
:10E720001FA1FEF7DFFD019800F016F9002815D1B2
:10E73000BE7002E0B878002814D026497A68B8681C
:10E7400000F076F8002809D1B87800280AD02246CF
:10E750002846059900F06CF8002803D00321397091
:10E7600007B0F0BD7878012804D0022805D003282E
:10E7700010D105E01F20800204E07F20800201E02C
:10E780001548C0682919814204D30220387010202E
:10E7900007B0F0BD002007B0F0BD0000A8F0FF1FDB
:10E7A0002E2E5C2E2E5C2E2E5C736F757263655C54
:10E7B0006461706C696E6B5C647261672D6E2D6450
:10E7C000726F705C666C6173685F6465636F6465CB
:10E7D000722E6300C8FBFF1FE4F1FF1F10B5EFF3BB
:10E7E0001081CC07E40F72B6FAF74EFF002C00D16F
:10E7F00062B610BD002801D10420704710B5144640
:10E8000000226260A260E26022616261A261E26154
:10E810002160C168616081684068FAF758F8A060BB
:10E820000420E06020616061A061E061002010BD13
:10E83000F7B53A4F0446787800261546012805D0EA
:10E840007B2237A10020FEF74DFD09E07869844264
:10E8500009D2832232A10020FEF744FD0220787005
:10E86000022003B0F0BDF878002809D1204602F05C
:10E87000C3F8060002D00220787011E00120F87081
:10E88000264FBA6878688118A14219D8B97800294A
:10E890000BD1B9698B682F49984706001CD102E05B
:10E8A000304603B0F0BD0120B870FF222948B96896
:10E8B000F9F7E4FF2046B968FAF709F8601A7860BA
:10E8C000002D28D03969F8684018A04208D82046A1
:10E8D00002F092F8060003D0104902204870DFE7EA
:10E8E0000E4948688968201A0F1ABD4200D22F4687
:10E8F00018493A4608180199F9F734FF002F08D053
:10E9000000200649E41988700198C019ED1B019098
:10E91000B6E70120F5E701484461C1E7B8F0FF1F01
:10E920002E2E5C2E2E5C2E2E5C736F757263655CD2
:10E930006461706C696E6B5C647261672D6E2D64CE
:10E94000726F705C666C6173685F6D616E61676544
:10E95000722E6300F8FBFF1F70B5274D04466878E0
:10E96000002806D0472225A10020FEF7BBFC02208C
:10E9700070BD002C2CD06068002829D0A068002829
:10E9800026D0E068002823D02069002820D06069C4
:10E9900000281DD0A06900281AD0E069002817D0EF
:10E9A0000121FF2289022248F9F768FF0126AE7093
:10E9B0000020E8706860A860E8602861AC61686168
:10E9C000206880470400D3D12878002807D010E0C1
:10E9D0004D220AA10020FEF785FC022070BDA86927
:10E9E00000698047040004D0A86940688047204639
:10E9F00070BD6E70FBE70000B8F0FF1F2E2E5C2E7E
:10EA00002E5C2E2E5C736F757263655C6461706C36
:10EA1000696E6B5C647261672D6E2D64726F705CE1
:10EA2000666C6173685F6D616E616765722E63000D
:10EA3000F8FBFF1F70B5194C00256178002902D042
:10EA4000012907D010E0CE2215A10020FEF74AFCD4
:10EA5000022070BDA078002806D1A0691D498368F6
:10EA6000A268606898470546A069406880470646E6
:10EA70000121FF2289021748F9F700FF0120002138
:10EA8000A070E1706160A160E1602161616161700D
:10EA9000002E01D0304670BD284670BDB8F0FF1F73
:10EAA0002E2E5C2E2E5C2E2E5C736F757263655C51
:10EAB0006461706C696E6B5C647261672D6E2D644D
:10EAC000726F705C666C6173685F6D616E616765C3
:10EAD000722E6300F8FBFF1F10B5EFF31083DC0705
:10EAE000E40F72B6FBF776FA002C00D162B610BDC7
:10EAF0008021017001780906FCD57047704700003D
:10EB0000024800698007C017401C704740F00F4062
:10EB100000207047174881B0816B1F2252021143B9
:10EB2000816315498015086108610861134A5060C6
:10EB300088601348102141604160416003680422ED
:10EB40001343036043690B43436143690B434361D0
:10EB500043690B434361416911434161094841697C
:10EB600002229143416108480090401E0090FCD170
:10EB700001B070470080044000C0044000A0044081
:10EB8000C0F00F4040F00F4040420F0070470000BF
:10EB900010220349012801D04A6070478A607047FB
:10EBA000C0F00F4010220349012801D04A6070478D
:10EBB0008A607047C0F00F4010220349012801D03D
:10EBC0004A6070478A607047C0F00F4010B50C4C27
:10EBD000A068002812D0401EA06020690949800169
:10EBE00041184022002003F0F9FB20690521401C58
:10EBF000F9F76DFE21616068401C606010BD000087
:10EC000008F0FF1F30F3FF1F70B50F4C002060604D
:10EC1000A060E0600D492061FEF704FF6060012004
:10EC20000B49C003FEF7FEFE0125A060AD021F20C8
:10EC300029468002FEF7F6FEE0607F20294680022A
:10EC4000FEF7F0FE206170BD40F0FF1FFC7B00006E
:10EC5000FC7B01000048704754F0FF1F0021064B69
:10EC60000A6A01209A4200D00020496A034A914270
:10EC700000D0002070470000939D939B01999697C8
:10EC80000021084B0A6A01209A4200D00020064B5E
:10EC90004A6A9A4203D1002801D0886A704700204E
:10ECA00070470000939D939B019996970148406897
:10ECB0007047000040F0FF1F014880687047000067
:10ECC00040F0FF1F0048704710F5FF1F00487047D5
:10ECD000CEF4FF1F0120C103054B0A6A9A4200D0FF
:10ECE0000020496A034A914200D00020704700008A
:10ECF0008F9E939B019996970120C103074B0A6A47
:10ED00009A4200D00020064B4A6A9A4203D100285A
:10ED100001D0886A70470020704700008F9E939B47
:10ED20000199969700487047C1F4FF1F004870474B
:10ED3000EFF4FF1F0048704790F4FF1F0048704732
:10ED400019F5FF1F0048704759F0FF1FF8B5FFF78E
:10ED50005BFF3F4800F0C6FF00243E4F2546264695
:10ED600021213D483C60F9F7AEFD21213B48F9F7F0
:10ED7000AAFD3B48FEF762FA3E71374E3448A100C7
:10ED80004158701903F094FC4019641CE4B2C5B2F8
:10ED9000042CF3D300207055304E0446054631480C
:10EDA000A9004158301903F083FC00196D1CEDB225
:10EDB000C4B2042DF3D300253555294C2A4E2046E4
:10EDC000316803F075FCC0B225542848006801780A
:10EDD0003175417871758178B175C078F0752448C6
:10EDE0003D71302101703221417035218170312116
:10EDF000C170057103261F48F9F767FD15491D48C5
:10EE0000F9F7A4FC1CA11B48F9F7A0FC124919480A
:10EE1000F9F79CFC21461748F9F798FC002415489F
:10EE2000F9F7CAFAC1B24800154A801C10700220D6
:10EE3000567000290BD90F4B1E5D1654401CC0B2F2
:10EE40001554401C641CE4B2C0B28C42F4D3F8BD2B
:10EE500070F4FF1F54F0FF1FCEF4FF1FEFF4FF1FED
:10EE600010F5FF1F80F4FF1F40F0FF1F00F0FF1F91
:10EE700059F0FF1F90F4FF1F3030303000000000C9
:10EE800019F5FF1F10B5134C2078002806D0632217
:10EE900011A10020FEF726FA022010BD0022114623
:10EEA0001046FBF751F8002801D01A2010BD0020B1
:10EEB0006070A070E070A060E0602071206160610F
:10EEC0000121A06189021248F9F7FDFC01202070A0
:10EED000002010BDD4F0FF1F2E2E5C2E2E5C2E2E97
:10EEE0005C736F757263655C6461706C696E6B5C9A
:10EEF000647261672D6E2D64726F705C6961705F02
:10EF0000666C6173685F696E74662E630000000052
:10EF1000F8FFFF1F0023002A0AD930B4DD000C4699
:10EF2000EC40C4545B1CDBB29342F7D330BC704757
:10EF30007047000002468800064910B54018803826
:10EF4000C06F002804D0114601F0F0F901F0DEF99D
:10EF500010BD0000B4FAFF1F80B501200749C003AF
:10EF6000886001F02BFCF9F7F5F8084F044A0549D1
:10EF70000548BC4600DF002080BD000000ED00E039
:10EF800008F6FF1F0A200300F9EF00000D0501003D
:10EF9000024901224A7008717047000060F0FF1FAB
:10EFA000024901220A70C8707047000060F0FF1F1C
:10EFB000024901228A7048717047000060F0FF1F0B
:10EFC00090B40448044F81680120C002BC4600DFB1
:10EFD00090BC704760F0FF1F41FF000090B40448F0
:10EFE000044F81680420BC4600DF90BC70470000DD
:10EFF00060F0FF1F41FF0000012086B0019006462F
:10F000000090162002900020A84F0546BC460390B1
:10F0100000DFA74CAA4FA0600023A64AA649A74834
:10F02000BC4600DFFEF77CFBFEF77FF9FFF772FDC1
:10F030000198FFF7B7FD0098FFF7AAFD3046FFF7EC
:10F04000BBFDFAF7EBFA00F0DBFA00F005FBFFF787
:10F050007DFE9D4F00229B490820BC4600DF03F047
:10F06000EBFF03F081FA012003F0D6FE002003F04D
:10F0700083F90120E0710B200490934F0022914905
:10F080009248BC4600DF924FBC4600DF0446800534
:10F0900009D587488079002803D08E4F0120BC46CF
:10F0A00000DFFCF70FFE600702D5022002F0EEFC45
:10F0B000E00612D5032002F0E9FC0020FFF766FD10
:10F0C000002003F059F90020FFF76CFD0020FFF746
:10F0D0005FFD0020FFF770FDFEE7A00602D50320CC
:10F0E00002F0D4FC200501D5FEF754F9E00735D035
:10F0F0005A2003F0DBFE6E4FF87900282ED001284D
:10F100000BD0032817D0052828D10020F871FFF76D
:10F110003DFD002003F030F920E00498002802D0E3
:10F12000401E04901AD1012003F026F90320F87143
:10F130001620029012E003F017F9002805D00120F4
:10F14000FFF724FD0220F87108E00298002802D0A1
:10F15000401E029002D10120FFF718FD200614D5B1
:10F1600001F030FB00285248816804D05A4F8020BB
:10F17000BC4600DF03E0594F8020BC4600DF4C480E
:10F18000554F81688020BC4600DFA00700D474E79B
:10F190000398002846D0FFF7B3FC002851D0FFF7B2
:10F1A000AFFC002810D04E4885420DD21E35ADB2BE
:10F1B000854209D101F0EEFB002805D03C48464FBE
:10F1C00081688020BC4600DF394C207800280BD0B5
:10F1D000E07801283FD002283DD001200190002096
:10F1E00020700198FFF7DEFCA07800280AD0607933
:10F1F00001283FD002283DD001260020A0703046D3
:10F20000FFF7DAFC60780028C1D0207901283ED0D1
:10F2100002283CD001200090002060700098FFF789
:10F22000B7FC2AE7FFF76CFC0028CDD02D4800681A
:10F23000C06980470028C7D102F028FC0120039054
:10F24000C2E72748854202D2022002F01FFC0020BC
:10F2500005460390B8E70199012901D0012100E09A
:10F26000002101910029BCD00128BAD100202070D2
:10F27000E070B6E7012E01D0012600E00026002E46
:10F28000BDD00128BBD10020A0706071B7E7009904
:10F29000012901D0012100E0002100910029BDD009
:10F2A0000128BBD1002060702071B7E7AD070100D5
:10F2B00060F0FF1F80F5FF1F0B880000991A010006
:10F2C000FD060100FFFF00009DFF0000B70A0000DF
:10F2D000E9FE0000C1FE000041FF0000CDFE00007D
:10F2E000B80B0000FC39010001498871704700002B
:10F2F00060F0FF1F10B5FFF77FF910BD10B5FF21BB
:10F3000004460231F9F7DFFA00F016FD0020207004
:10F31000FFF772F910BD000001280BD002280FD0B2
:10F32000032813D0D1220CA10020FDF7DBFFFBF74F
:10F3300061F9FEE7C52208A10020FDF7D3FFF6E73B
:10F34000C92205A10020FDF7CDFFF0E7CD2202A1E3
:10F350000020FDF7C7FFEAE72E2E5C2E2E5C2E2E36
:10F360005C736F757263655C6461706C696E6B5C15
:10F370005254585F436F6E6669672E630000000049
:10F38000FEE70000074801680748416100218161EC
:10F39000072101610548016AFF221206114301623B
:10F3A00040177047C039010000E000E000ED00E0C8
:10F3B00070477047FFB583B0054604980E9C2F1820
:10F3C0000020206089488A4EC07800281ED08748D7
:10F3D0000021C1708748884902780698F9F7C2F978
:10F3E000701E00780699411806912168081820605F
:10F3F0007E48717840683278000C0902000411439D
:10F400000843711E0978411878484160BD426ED0AA
:10F4100028780A280CD00D280AD03A2868D07349D9
:10F420000A78002A7ED0C2067DD50007000FA7E02B
:10F43000704A0021137801939C4608465B1D0DD04D
:10F4400063465B1D9C46135C401C5918C0B2C9B290
:10F450008445F8D8002901D00426B2E063488178B9
:10F46000002941D101218170707831780002084370
:10F4700040BA3070010A717000905E48C078002870
:10F4800006D0012831D0022833D004282CD14DE0F9
:10F49000252258495948F9F765F95448009A4068B7
:10F4A000010C09041143814204D001204F49022676
:10F4B000C87086E05049019A0698F9F753F94D480B
:10F4C00006990078494B4118069121680818206078
:10F4D000586871783278000C09020004114308431F
:10F4E000444909784118596066E0012669E067E0FF
:10F4F00039E021680C98FF22411A0698F9F7BEF905
:10F500003A4920684A68121A0D98026004987A1BDA
:10F51000821A059802603748027940791203000187
:10F52000024301E038E028E04A6019E021680C98C5
:10F53000FF22411A0698F9F7A1F92C4920684A6878
:10F54000121A0D98026004987A1B821A05980260BC
:10F550002848427903791002184340BA00044860F1
:10F56000022007B0F0BD25212248F9F7ACF91F4869
:10F5700000210170417081701EE00007000F09300A
:10F5800002071C4B4878120F1B5C1A43194B1A5484
:10F59000401C487000200EE04A78252A0AD2C30693
:10F5A00002D50007000F02E00007000F0930114BE1
:10F5B00000019854012008706D1CBD4200D027E75F
:10F5C000002621680C98FF22411A0698F9F756F98F
:10F5D000064821684068411A0D9801600498791B1B
:10F5E000411A05980160304607B0F0BDF0F0FF1FEA
:10F5F000F9030020F8030020FC0300201D04002074
:10F60000FF20104A81B0033010600F49486940085C
:10F61000400048610D480090401E0090FCD10869F0
:10F62000C007C00F0021116009490A4A002802D012
:10F63000486804D000E00868106001B070471060AE
:10F6400001B0704700A0044040F00F4010270000B8
:10F650001039010000F0FF1F7047000070B5134D16
:10F660000646EFF31080C407E40F72B62846FAF797
:10F670000BF8002C00D162B6002816D1FF22102111
:10F680000B48F9F7FBF8092231460948F9F76AF8FF
:10F69000EFF31080C407E40F72B6054A1021284624
:10F6A000FAF798FC002C00D162B670BD00FC010096
:10F6B000B0250020F7B504461F2084B080028C4E90
:10F6C000029030781546012805D0A32289A1002098
:10F6D000FDF708FE61E0FF2101318F002046009117
:10F6E000F9F7F5F8002908D0AC2282A10020FDF737
:10F6F000F9FD0220307007B0F0BD0098854205D3B7
:10F7000001462846F9F7E3F8002908D0B32279A189
:10F710000020FDF7E7FD0220307007B0F0BD39464C
:10F720002046F9F7D4F84819B84208D9BA2271A18D
:10F730000020FDF7D7FD0220307007B0F0BDB07893
:10F7400000281BD1F07800280FD0B068844203D382
:10F75000F1684018A04211D8C82266A10020FDF728
:10F76000C1FD0220307007B0F0BDC22261A10020AF
:10F77000FDF7B8FD0220307007B0F0BD30790028E9
:10F780000ED0716930694018A04209D0D02259A129
:10F790000020FDF7A7FD02203070022007B0F0BD69
:10F7A0007F2080026719844207D20120C00387426C
:10F7B00003D90020002810D002E0012000280CD03E
:10F7C00001214B481F260171456104610598B6026D
:10F7D0000190B44204D31F2667E00220307079E024
:10F7E000FEF78AF900285FD0301B0090001F2946E1
:10F7F000A84201D90A4601E0009A121F3C4801992B
:10F800008069FEF741F93A49844688610120800207
:10F81000844207D245492A4608190199F8F7A2FF00
:10F82000002642E0B7423FD1019900980B181C20F6
:10F83000203B19180A7810464A78120210438A7839
:10F84000C9781204104309060843D97F0002000A50
:10F8500009060843844501D0232626E02946204690
:10F86000019AFFF739F9002801D01C261DE000207D
:10F8700000902E4801260190B6020098FEF7AEFFD8
:10F88000002801D00E2609E03146019A0098FFF7C2
:10F8900023F9002801D01C2600E00026FFF7B4F968
:10F8A00013490120487000E022263046222E07D05E
:10F8B000002800D172E70E4A0221117007B0F0BD96
:10F8C00029462046059AFFF707F9002805D0084980
:10F8D000022008701C2007B0F0BD0298874204D3B4
:10F8E000FFF792F9024901204870002007B0F0BDEF
:10F8F000D4F0FF1F2E2E5C2E2E5C2E2E5C736F75A7
:10F900007263655C6461706C696E6B5C6472616784
:10F910002D6E2D64726F705C6961705F666C6173CF
:10F92000685F696E74662E6300000000F8FFFF1FB9
:10F93000FF2001307047000070B514460E460546A2
:10F940000019012140028902884206D90B4A0CA104
:10F950000020FDF7C7FC002070BD012149023046A0
:10F96000F8F7B1FF002D06D1124813494069420152
:10F970003046F8F7F7FE600270BD0000A6030000F5
:10F980002E2E5C2E2E5C2E2E5C736F757263655C62
:10F990006461706C696E6B5C647261672D6E2D645E
:10F9A000726F705C7669727475616C5F66732E63DA
:10F9B0000000000010F1FF1F3C10002010B50124D2
:10F9C00064020B46002801D0002010BD22460349E6
:10F9D0001846F8F7C7FE204610BD0000BC0C0020FA
:10F9E000F8B50C4600210E460091002801D00020F9
:10F9F000F8BD33480078012845D0022845D00027BB
:10FA000030A1204602F07EFE0546601930A102F0CA
:10FA100079FE45196019304902F074FE45196019E4
:10FA20002EA102F06FFE451960192DA102F06AFEA9
:10FA3000234945196019498802F070FE451960197B
:10FA400026A102F05FFE4519002F0ED0601926A1F5
:10FA500002F058FE45196019394602F053FE451967
:10FA600060191EA102F04EFE45196846FDF720FF01
:10FA7000070022D0009800281FD060191DA102F0B5
:10FA800041FE451911E01EA7BAE720A7B8E7B0006C
:10FA90000099761C0958F6B2601902F009FE451962
:10FAA00060190EA102F02EFE4519BE4205D228466D
:10FAB00001210A3049028842E9D32846F8BD0000F6
:10FAC00004F1FF1F4173736572740D0A000000009A
:10FAD00046696C653A200000780800200D0A000095
:10FAE0004C696E653A200000536F757263653A2069
:10FAF0000000000048657864756D70730D0A0000A1
:10FB0000426F6F746C6F6164657200004170706C5D
:10FB100069636174696F6E00002801D0002070472E
:10FB2000084610B50121490202F00CFA10BD000090
:10FB3000F8B50D46044603F0B1F90746FEF7D4F8D0
:10FB400006463846FEF7F4F80746002C01D00020A0
:10FB5000F8BD1B49284602F0D5FD04462819314658
:10FB600002F0D0FD0419281916A102F0CBFD0419EA
:10FB70002819154902F0C6FD04190026012000903D
:10FB800014E00098002804D1281910A102F0BAFD51
:10FB90000419F80708D00E48B1004158281902F09E
:10FBA000B1FD0419002000907F08761C002F01D0C1
:10FBB000052EE6D3281903A102F0A4FD0019F8BD13
:10FBC000673A01000D0A0000603A01002C20000095
:10FBD0006C3B010010B50B46410254022246184608
:10FBE00003F034FA204610BD10B50B464102540212
:10FBF0002246184603F02EFA204610BD002801D0F8
:10FC00000020704770B50C4601256D02294620463C
:10FC1000F8F759FE0648F8F7CFFB0246044920469C
:10FC2000F8F7A0FD29462046FEF78CF870BD0000CD
:10FC30006F3A0100F8B5094D04460E462846F8F71C
:10FC4000BBFB0746002C01D00020F8BD0246294628
:10FC50003046F8F787FD3846F8BD00005C4A0100E1
:10FC600010B50B46410254022246184603F0EEF945
:10FC7000204610BD10B50B465202410214461846EC
:10FC800003F0E8F9204610BD10B50B4641025402BE
:10FC90002246184603F0E6F9204610BD10B50124AF
:10FCA00064020B46002801D0002010BD2246034903
:10FCB0001846F8F757FD204610BD0000BC0A00208A
:10FCC00010B5012464020B46002801D0002010BDAD
:10FCD000224603491846F8F745FD204610BD0000AE
:10FCE000BC08002004490A6A0260CA694260896946
:10FCF00081600021C16070474080044010B5084613
:10FD000054022146F8F7DFFD204610BD70B40023F1
:10FD10001A4600290CD90125C40704D08E1A2C4696
:10FD2000761EB4402343521C4008D2B28A42F3D319
:10FD300070BC18467047000010B525210748F8F739
:10FD4000C2FD25210648F8F7BEFD064800214160A6
:10FD5000017041708170C17010BD0000F803002077
:10FD60001D040020F0F0FF1F0146EFF31080C207D2
:10FD7000D20F72B60868002801D003680B60002A11
:10FD800000D162B670470000002813D070B50D4650
:10FD900009490A4C884204D222680146104600F004
:10FDA000E5FA20684570064800F029F902216060F4
:10FDB000417070BD70470000FFFF0000D0F1FF1FD1
:10FDC000B824002070470000F0B4284FF8680028DD
:10FDD00049D0B88A401EB88200263EE081680029DA
:10FDE00008D042684A604168002902D082688A606F
:10FDF000466086601E4A00251178022903D0012939
:10FE000001D0032900D10125837800E00A4651681A
:10FE1000002902D08C789C42F8D241605060002DBD
:10FE200004D0002900D08860826000E08660818A6A
:10FE3000B9824178042904D10E49C28A098851182F
:10FE400081820121417020221154C168F960C1688A
:10FE5000002901D00F61C6600661B88A002802D16E
:10FE6000F8680028BAD1F0BC70470000D024002008
:10FE7000B8240020D8F1FF1FF8B502260E4D044625
:10FE800000280CD02868A1788278012791420CD9EB
:10FE900000F0BAFA286847706C606670F8BD0748D1
:10FEA00000F0ADF868604670F8BD67702146034801
:10FEB00000F088FAF8BD0000D0F1FF1FB824002040
:10FEC00010B50321FFF760FF10BD0000054A89004F
:10FED00089188039C96F002902D00A8B82430A83AE
:10FEE00070470000B4FAFF1F01480068408B70475C
:10FEF000D0F1FF1F10B50446008B084320836278C1
:10FF0000618B062A15D0052A12D1084210D00A4664
:10FF10000240628388432083204600F0ABFA012030
:10FF200060700221202001552146044800F04AFA61
:10FF300010BD0A468243EDD010BD0000B824002059
:10FF40000246880070B5144940188038C46F002CF0
:10FF50001DD0208B104320836178658B062917D034
:10FF6000052914D1284212D0294601406183A843B3
:10FF70002083204600F07EFA208B0221A8432083B4
:10FF800001206070202001552046FFF775FF70BDED
:10FF900029468143EBD070BDB4FAFF1F10B50C4663
:10FFA0000C49002A0B68198B08D002468A4301D0FD
:10FFB000062109E081431983022010BD0A46024050
:10FFC00001D05A83F6E7052158832046FFF7DCFE6F
:10FFD000012010BDD0F1FF1F814202D342688A4246
:10FFE00001D801207047EFF31082D207D20F72B60A
:10FFF00003680B60016000D162B6002070470146C3
:020000040001F9
:100000004068002342684A600A78022A05D0012A23
:1000100003D0032A01D0436070474268002A01D010
:1000200091604360836070477047000030B4428C39
:10003000920803D10F4A12881204920C836A92002C
:100040009B185A0700D51B1F01221206403BDA639A
:100050000022996314469500521C5C510E2AFAD373
:10006000C2691A624362C162806A0349016030BC9E
:1000700070470000BC390100A52E5AE20349044A2A
:100080000968C8821288801888827047D0F1FF1FE3
:10009000D8F1FF1F0848016808488A8A0088CB8A7F
:1000A000101AD21880B28A82010404D410B5042137
:1000B000FFF76AFE10BD7047D0F1FF1FD8F1FF1F98
:1000C000F8B50446406800260F46002805D0607841
:1000D000022818D0A08900282FD0A089E189884261
:1000E0003ED2208980000019076172B6A089401CA9
:1000F000A08162B62089401C80B22081E1898842BB
:1001000000D12681F8BD66702046FFF778FF0546CE
:10011000203006702189E86989000919086172B6E2
:10012000A089401CA08162B62089401C80B2208139
:10013000E18988420AD1268108E02046FFF75FFF67
:100140000546C069042107602020415501206870E0
:10015000284600F08FF92946034800F033F9F8BD2E
:100160000320FFF7D9F8F8BDB8240020032101705F
:10017000002141704180416081607047F8B50446BC
:100180004088002804D0264EA1683268914201D0F0
:10019000FF20F8BD401E0004000C60803ED1316895
:1001A0006078887061680127002928D02046FFF711
:1001B00026FF0546052120300170284600F05AF937
:1001C0006780A560A87860701648316840688A78B2
:1001D0008078824201D328460AE0124800F0F2F803
:1001E0002946104800F0EEF8306847706F70002024
:1001F000FFF742FE31680020203108700EE0094907
:1002000049688A783168824208D9064800F0DAF8ED
:10021000306847700020FFF72FFEEBE70020F8BDA5
:10022000D0F1FF1FB824002070B50E46194D0446CA
:1002300041882868002907D0A168814208D16088D8
:10024000401C6080002070BDA06080786070F6E780
:10025000002E0FD062788078824203D28870A06826
:1002600000F0DCF86068002806D02046296800F01D
:10027000A9F808E0012070BD2868606029680020A6
:1002800048602868846009213046FFF77DFD012021
:1002900070BD0000D0F1FF1F70B519480121026840
:1002A0005170006800F0B0F8164DA8786C780028FE
:1002B00016D0E000411948680278002A17D0012AB8
:1002C0001AD000F0EDF8E878641C844200D10024D4
:1002D00072B6A878401E0006000EA87062B6E8D17B
:1002E0006C700948FFF78BFE00F008F970BD0989B2
:1002F00089B2FFF7FFFDE6E78968FFF7E1FEE2E775
:10030000D0F1FF1F90FAFF1FB824002005480178A4
:10031000002902D0012141707047012002490007E5
:1003200048607047C8F1FF1F00ED00E0F8B50E4EC1
:10033000F778B41C354672B6B278BA4207D2521C6E
:1003400022702A78531CBB4200D100232B7062B666
:10035000F378934204D9D200921991605060F8BDAD
:100360000220FEF7D9FFF8BD90FAFF1F10B4144A1F
:10037000D368002B1BD013469B8A8B4203D307E024
:10038000D468002C13D0D268948AE3188B42F7D338
:10039000D468C460D0600261C468002C00D02061C1
:1003A000591A8182908A401A908210BC70470024AA
:1003B000C460D060C91A02619182848210BC704707
:1003C000D024002030B402780023022A03D0012A6E
:1003D00001D0032A00D101238C7800E01046426846
:1003E000002A02D09578A542F8D24A604160002BDD
:1003F00005D0002A00D09160886030BC7047002092
:10040000886030BC7047000003494A68426000229F
:100410008260486070470000B824002010B58368EF
:100420000146002B04D01A781846002A05D008E0AF
:10043000487801281AD10E4803E080680278002A23
:10044000FBD0002B07D04A685A604A68002A0BD0BC
:100450008B68936008E0064A53688B4202D14B6870
:10046000536001E01A00F7D1FFF7ACFF10BD0000A8
:10047000B824002010B4016900290FD0C268CA60F6
:10048000C3680022002B07D08B8A848A1B198B82B9
:10049000C3681961C26000E08A82026110BC7047C3
:1004A00010B5416800290ED0FFF7A9FD0446FFF7FB
:1004B000E1FF0120607003212020015521460448FE
:1004C000FFF780FF10BD4188491C418010BD00002E
:1004D000B824002007480068416A806A814203D33B
:1004E00000680549884204D010B50120FEF714FFCA
:1004F00010BD7047D0F1FF1FA52E5AE20249486097
:100500000221417070470000D0F1FF1FF7B5454947
:1005100000200A8882B00546002A05D94249830096
:10052000401CCD509042FAD34048302201884048C8
:10053000FCF794FE3F4801210088C90780B24218A9
:100540003D4801683D48FCF789FE3D480822018886
:100550003C480068FCF782FE3B4EFF20F07075843B
:100560003A4834460090257001276770A570656091
:10057000A560E5602561A582E58225832046658327
:100580002030057045702D48FFF7EEFBA062204635
:100590000099FFF74BFD2E480421017045602D485E
:1005A0000170C56005618582706A2030F7F7CCFD67
:1005B00029482B4906600220707028480570457054
:1005C0000978C170FFF730FD2648016AFF22120446
:1005D00011430162C169026A5202920E92061143EE
:1005E000C161FEF7CFFE20490028086012DB8208B7
:1005F0001E49920051180B688207D40EFF22A240B8
:1006000013430B60C106C90E8F404011184980008A
:10061000401807600023049A0399029800F06EF8CE
:1006200005B0F0BDB8390100B4FAFF1FD0390100A0
:1006300028F9FF1FBC390100D4390100F8F9FF1F68
:10064000DA3901006CF0FF1FE824002081F300007C
:10065000B8240020D0240020D0F1FF1F90FAFF1F03
:10066000D839010000ED00E0CCF1FF1F00E400E00C
:1006700000E100E010B50B480121026851700068EC
:10068000FFF7C2FEFFF79EFB07480168491C0160A7
:10069000FFF79AFB00F012F80448FFF7B0FCFFF7F1
:1006A0002DFF10BDD0F1FF1FD8F1FF1FB82400208F
:1006B0000148006870470000D8F1FF1F70B50D4D6C
:1006C0002868002815D0A8880B4E401EA8800AE094
:1006D000E088FEF76EFEA088A8802068286021468A
:1006E0003068FFF779FCA888002802D12C68002C1C
:1006F000EED170BDDCF1FF1F6CF0FF1FFFB50746A8
:10070000080681B016460D46000E00D14D1C224849
:10071000FFF72AFB041E3DD02802A662000C60846D
:100720000499E1610026267001216170A570666060
:10073000A660E6602661A682E682214626832031F5
:1007400066830E704E70002803D11448FFF70CFB2F
:10075000A06239462046FFF769FC1148012501884F
:10076000104A012908D3A80080188038C06F0028DB
:1007700003D06D1C8D42F6D93546A800801880380C
:10078000C467E5702046FFF777FB07480068203014
:100790000570284605B0F0BD28F9FF1FF8F9FF1FC6
:1007A000B8390100B4FAFF1FD0F1FF1F02480068FA
:1007B000002800D0C0787047D0F1FF1F704700209C
:1007C0007047000070B5334C0026E07800285FD0F9
:1007D0002089A1880025884250D2E0882E4A904284
:1007E00049D2022847D30120FEF7DAFB01216069D4
:1007F000090388422AD22169E268CB1DF93393426A
:1008000012D2A169FF25091801352A46234802F0B2
:1008100029FC2946214800F0C7FA206940192061C7
:1008200060694019606127E0521AA16909181B48E4
:1008300002F018FC2169E068411A184800F0B4FA87
:10084000E0682061A0882081656115E0E0880222CF
:100850004100124802F0FEFB104A50780102107865
:100860000843E0800E4900034018A0612089401C25
:100870002081656100E02181012609E0884207D1DD
:1008800000F0D0F9E5702089401C208101F098FA31
:10089000304670BD2CF1FF1FF0FF00004F15002007
:1008A00000E0FFFF70B50546002400F063FA06463D
:1008B00003281CD00F4A1049284602F01BF90028D3
:1008C00015D0304600F0F0F90C480D4AC168090116
:1008D0008918090C81800021018101614161C18871
:1008E000084A0903891881610121C1700C4620461C
:1008F00070BD000038F1FF1F32F1FF1F2CF1FF1F08
:10090000F0FF000000E0FFFF70B5204C21780029C7
:100910001DD0012552281BD021468A7849784128CC
:100920001ED0422826D0432801D053280FD10029B9
:100930000AD0002020700B204143154808180B38BE
:10094000FFF7B0FF002802D10D2000F043F870BD82
:1009500019210F4802F0FCF8A070002812D1F3E72B
:10096000012902D9491EC8B20DE0002AECD06270FC
:100970001046EAE7914203D2491CC8B26070E4E72E
:10098000002AE1D028466070DFE700002CF1FF1F4D
:100990003C14002010B5002409A0FFF783FF0028B5
:1009A0000BD00A4800214170817001210170FF21A4
:1009B00014310748F7F787FF0124204610BD0000D7
:1009C00053454C4543545220484558002CF1FF1FD5
:1009D0003C14002008B507A212686946009208700E
:1009E0000146684601F09AFE0321684601F04CFA80
:1009F00008BD0000000D0A00F1B5354DA869416938
:100A0000009888470746A869816900988847044686
:100A1000002F07D0002C05D00126B602B74209D816
:100A2000012008E0FF222A322AA10020FCF75AFC0C
:100A30000220F8BD0020FF222F3226A1FCF752FC35
:100A400039463046F7F743FF002909D00020FF223E
:100A5000303220A1FCF746FCBC4203D3012002E067
:100A60000120F4E70020FF2231321AA1FCF73AFC02
:100A700039462046F7F72BFF00291FD00020FF2220
:100A8000323214A1FCF72EFC21460098F7F71FFF25
:100A90000098401AE8602C616860B44200D3344684
:100AA000AC60297800290BD0A969C968884704007F
:100AB00006D0A869416888472046F8BD0120DEE7D6
:100AC000FF221148A968F7F7D9FE0020F8BD000001
:100AD000B8F0FF1F2E2E5C2E2E5C2E2E5C736F75D1
:100AE0007263655C6461706C696E6B5C6472616793
:100AF0002D6E2D64726F705C666C6173685F6D61E2
:100B00006E616765722E6300F8FBFF1F01490420C8
:100B10004860704780F00F400149042088607047AA
:100B200080F00F40F0B4FF2014490430C861144A2B
:100B3000C01E90615061134A10608860486012487E
:100B400041694022114341614169202529434161A6
:100B50000E4C61690126314361610D494A690427E0
:100B60003A434A614B69022213434B6166604F600E
:100B70004A60856040218160F0BC704700B004404D
:100B800000C0044000A00440C0F00F4040F00F40FF
:100B900080F00F40F0B4064600200E4C20250146A0
:100BA00007278022CA40324202D04022626001E020
:100BB0004022A2606560084A1269A5601206D20F41
:100BC0007B1A9A400243D0B2491C0829E9DBF0BCE9
:100BD00070470000C0F00F4080F00F40F0B40646B0
:100BE00000200E4C202501460F270122D203CA40C7
:100BF000324202D04022626001E04022A260656081
:100C0000074A1269A5601206D20F7B1A9A40024366
:100C100090B2491C1029E8DBF0BC7047C0F00F40CF
:100C200080F00F40B0B50F4C2078002807D00E4F51
:100C3000BC4600DFA168884208D1012007E0C1223C
:100C40000AA10020FCF74EFB0220B0BD0020632269
:100C50001349FCF747FB6068C168124888470021C8
:100C60002170B0BD7CF0FF1FAD0701002E2E5C2E61
:100C70002E5C2E2E5C736F757263655C6461706CA4
:100C8000696E6B5C647261672D6E2D64726F705C4F
:100C900066696C655F73747265616D2E6300000038
:100CA000540E0100C4FAFF1FB0B5164D0446287853
:100CB000002806D0862214A10020FCF713FB022096
:100CC000B0BD022C06D38C220FA10020FCF70AFB3A
:100CD0000220B0BD194FBC4600DFFF21A8600531DE
:100CE0001748F7F7F2FD0120287016492001401837
:100CF00068604168124888470028EAD003212970BB
:100D0000B0BD00007CF0FF1F2E2E5C2E2E5C2E2E20
:100D10005C736F757263655C6461706C696E6B5C4B
:100D2000647261672D6E2D64726F705C66696C65AC
:100D30005F73747265616D2E63000000AD07010082
:100D4000C4FAFF1F88F0FF1FF8B5094D0E4607468D
:100D5000002420012A58314638469047002801D007
:100D60002046F8BD641CE4B2022CF2D30320F8BD87
:100D700088F0FF1F014610B5083103220C4608A079
:100D8000F7F794FC002807D00322214605A0F7F7C7
:100D90008DFC002801D0032010BD012010BD0000F3
:100DA00042494E0048455800F8B51B4D0646287884
:100DB0000C46012806D0A52218A10020FCF792FAC3
:100DC0000220F8BD224FBC4600DFA968884201D14D
:100DD000012000E0002063221EA1FCF783FA68686E
:100DE000224683683146284898470446102807D091
:100DF000112C07D0002C05D0032028702046F8BD08
:100E00000220FAE72878012800D00020B32203A1AD
:100E1000FCF768FAF2E700007CF0FF1F2E2E5C2E34
:100E20002E5C2E2E5C736F757263655C6461706CF2
:100E3000696E6B5C647261672D6E2D64726F705C9D
:100E400066696C655F73747265616D2E6300000086
:100E5000AD0701002E2E5C2E2E5C2E2E5C736F755E
:100E60007263655C6461706C696E6B5C647261670F
:100E70002D6E2D64726F705C66696C655F73747241
:100E800065616D2E63000000C4FAFF1FFFB593B0CB
:100E900004461F46442168461D9E1C9DF7F715FD1C
:100EA0001598029501970396009060680990A068D4
:100EB0000D9020680E9014980F900120000610905D
:100EC0006D460021082000F0E7FB002853D00024E5
:100ED000A0002958204600F089FB00284BD0641C54
:100EE000042CF5D30920696A00F080FB002842D069
:100EF0000D24A0002958204600F078FB00283AD0A5
:100F0000641C102CF5D31020296C00F06FFB002816
:100F100031D01F4D1D49284600F064FC00282AD01E
:100F20001C49284600F05EFC002824D011A90420AA
:100F300000F048F900281ED01198A02108421AD1CB
:100F4000154E002411AF1549002000F021FB0028A8
:100F500011D03946284600F005F900280BD0119829
:100F600080030BD56946002000F0CAF8002803D0A2
:100F70000098002806D0002017B0F0BD641CB442D1
:100F8000E0D3F8E7012017B0F0BD00000B005FA030
:100F9000F0ED00E009005FA040420F005200002386
:100FA00010B5F8F73BFB0848202242604021416021
:100FB000416043691343436142690A4342614269A4
:100FC0000A434261012010BD80F00F40F8B50021B6
:100FD000C9433F486425016004264160002413E0B2
:100FE000002C11D00121002000F056FB012000F060
:100FF000AFF9384F0220BC4600DF002000F0A8F90E
:101000000220BC4600DFE9E7F8F708FB324820235E
:10101000436040214160416042691A434261426934
:101020000A43426142690A43426100F007FCF8F753
:10103000A3FF00282AD01E21002000F02DFB00284D
:1010400024D00021082000F027FB00281ED0052115
:101050000907042000F020FB002817D00027002DEE
:1010600022DD0620694600F083FA6A46D17892783C
:101070000906120411436A465278120211436A4665
:1010800012781143012808D001240DE0761E0124B6
:1010900076B2002EA4DC0020F8BD0520400788436E
:1010A00002D07F1CAF42DCDBAF42EFD0012CEDD091
:1010B0000A49042000F0F0FA0028E7D000F0EAFC2A
:1010C0000021082000F0E8FA0028DFD00120F8BD58
:1010D00070F0FF1FC1FE000080F00F40000F0050B5
:1010E00006484169202291434161426940218A4377
:1010F000426142698A4342610120704780F00F409B
:10110000F8B50D46014600246426124800F06AFB3B
:10111000002815D0104F1149002000F039FA00289E
:101120000DD02946384600F01DF8002807D0286861
:10113000C00302D4641CB442EDDBB44201D10020F0
:10114000F8BD2946064800F0EFF80028F8D0012045
:10115000F8BD0000F4ED00E0F0ED00E052000023E7
:10116000F8ED00E010B50C4682B00146042201A85B
:10117000FDF7D0FE052001A900F0FAF901281ED1E3
:101180000F20694600F0F4F9012818D10E206946B5
:1011900000F0EEF900216A462160D178090621604D
:1011A0009278120411436A46216052781202114368
:1011B0006A462160127811432160012800D0002086
:1011C00002B010BD38B50C460C2108406946801CA1
:1011D00000F0CEF900216A462160D178090621602D
:1011E0009278120411436A46216052781202114328
:1011F0006A462160127811432160012800D0002046
:1012000038BD0000F0B585B014460E46054613E023
:101210004349002000F0BCF900287DD069462846EB
:10122000FFF7A0FF002877D0A807C10E0098C8409C
:101230003070761C641E6D1C002C69D0A807E7D1A5
:10124000032C4CD9A9050120890D8002471ABC4204
:1012500001D2A708BF000096002F5DD0B808039008
:101260003049002000F094F9002855D00520019065
:101270000422294604A8FDF74DFE04A9019800F0B8
:1012800077F9012848D10F200021019000F070F972
:10129000012841D1002002900398012811D0039821
:1012A000401E03900099019800F062F9012833D1A3
:1012B00000980399001D00900298401C02908842FB
:1012C000F0D30E20009900F053F9012800D000203F
:1012D000002821D0ED19F619E41B032CB2D8002CFC
:1012E00016D00F4F0020394600F052F9002813D0D5
:1012F00069462846FFF736FF00280DD0A807C10E23
:101300000098C8403070761C641E6D1C002CE9D11A
:10131000012005B0F0BDFFE7002005B0F0BD0000E2
:10132000500000235200002370B50C4605460749C3
:10133000002000F02DF9002806D021462846FFF7AE
:1013400011FF002800D0012070BD000052000023D2
:1013500070B520250B4C4026002810D0FFF736FE34
:101360000949042000F014F9002807D001210C20BD
:1013700000F00EF9002801D0A560A66070BD656080
:10138000666070BD80F00F4044050040F8B502244F
:101390000746062801D0FFF703FE6C493846CF1CEC
:1013A0006B4D6C4E08287DD202007A441279921857
:1013B00097440317077F85A5C0C70120FFF7C8FF23
:1013C000BFE00120FFF7C4FF634F0220BC4600DFEF
:1013D0000020FFF7BDFF0220BC4600DFFFF780FEC4
:1013E000AFE0FFF7F3FD00287DD03946284600F036
:1013F000F9F9002816D1641E64B2002C52DD0120D8
:10140000FFF7A6FF544F0220BC4600DF0020FFF785
:101410009FFF0220BC4600DF5049284600F0E2F959
:101420000028E8D034466E462146002000F0B0F88F
:10143000002837D031462846FFF794FE002831D0E7
:1014400000988003EFD5464E0121304600F0CAF9DE
:10145000002877D0434F69463846FFF765FF0028DC
:1014600070D00098710D08403F494118384600F08F
:10147000B9F9002866D0384F0220BC4600DF274665
:101480006C463946002000F083F800285BD02146E6
:101490002846FFF767FE002855D000988003EFD557
:1014A000002100E04FE0304600F09CF9002849D0D0
:1014B00047E0284600F096F9002843D041E0F8F7CD
:1014C0005BFD00283ED01E21002000F0E5F800283A
:1014D00038D00021082000F0DFF8002832D00521A4
:1014E0000907042000E02DE000F0D6F8002829D0FC
:1014F0001E49284600F076F9002823D021E0FFF7A6
:1015000065FD00281ED03946284600F06BF90028FA
:1015100018D06C463146002000F03AF8002812D06E
:1015200021462846FFF71EFE00280CD000988003B5
:10153000EFD506E0284600F055F9002802D0FFF765
:10154000CFFD0120F8BD0020F8BD000000005FA025
:10155000F0ED00E052000023C1FE000003005FA098
:10156000FCED00E00CED00E00400FA0501005FA0D6
:1015700070B50D460646002429463046F8F74CFD66
:10158000022803D1641CE4B2642CF5D370BD0000C2
:1015900038B50D46010E0446F022090610400143FD
:1015A000082000F079F8002806D0002C06D10E485B
:1015B0004168A94201D1012038BD45600C2004409A
:1015C000042229466846641CFDF7A4FC69462046AF
:1015D000FFF7CEFF012805D10E200021FFF7C8FF3D
:1015E0000128E9D0002038BD70F0FF1FF3B581B0AD
:1015F0000546002464261448029900F0F3F80028F8
:101600001AD00120000405432946104800F0EAF8EA
:10161000002811D00E4D02AF0E490020FFF7B8FF91
:1016200000280ED039462846FFF79CFD002808D038
:101630000298C00302D5012003B0F0BD641CB4427F
:10164000E9DB002003B0F0BDF8ED00E0F4ED00E0D0
:10165000F0ED00E05200002338B50C4601460422AC
:101660006846FDF757FC05206946FFF781FF012812
:1016700010D1042221466846FDF74CFC0D20694636
:10168000FFF776FF012805D10E200021FFF770FF3C
:10169000012800D0002038BDF8B50E4F04460D4695
:1016A000082802D13868A84211D00C2026460640EE
:1016B00004226846FDF72EFC69463046FFF758FFC6
:1016C000012801D00020F8BD082C00D13D60012088
:1016D000F8BD000070F0FF1FF0B585B014460E464F
:1016E000054612E037783D490020FFF751FF0028FA
:1016F00071D0A807C00E394681402846FFF7ACFFDD
:10170000002868D0641E6D1C761C002C5FD0A807D2
:10171000E8D1032C44D9A9050120890D8002471A7C
:10172000BC4201D2A708BF000096002F53D0B808D2
:1017300003902B490020FFF72BFF00284BD00520FA
:1017400001900422294604A8FDF7E4FB04A90198AE
:10175000FFF70EFF01283ED10D20019000200290DE
:10176000039800280ED900990198FFF701FF01287E
:1017700031D100980399001D00900298401C0290FE
:101780008842F0D30E200021FFF7F2FE012800D09E
:10179000002000281FD0ED19F619E41B032CBAD83D
:1017A000002C14D037780D490020FFF7F1FE0028F7
:1017B00011D0A807C00E394681402846FFF74CFFDC
:1017C000002808D0641E6D1C761C002CEAD1012074
:1017D00005B0F0BDFFE7002005B0F0BD50000023CC
:1017E0005200002370B50C46054607490020FFF75C
:1017F000CFFE002806D021462846FFF72DFF0028FF
:1018000000D0012070BD00005200002380B5084FB9
:10181000BC4600DF07494968884201D1012000E049
:101820000020FF2283320449FBF75CFD80BD0000ED
:10183000AD070100F8F0FF1FEC2F0100704700001A
:1018400002480078012800D00020704778F0FF1F80
:1018500002480078012800D000207047D4F0FF1F14
:1018600030B500250C4C83B0A069009501958168C6
:101870002B462A461830FFF709FB002808D0207FA6
:10188000002802D000F044F80546284603B030BDD9
:101890000E2003B030BD0000E4F1FF1F30B5054657
:1018A0000E4883B08469284600F01AF8014628469D
:1018B000F7F70DF800290ED10020009001900346A3
:1018C00020462A461830E168FFF7E0FA002802D0E7
:1018D000002003B030BD0D2003B030BDE4F1FF1F88
:1018E00010B40A4B596A00290DDD491E0BD41A6A3F
:1018F000CC001459844204D8C800001D105810BCF4
:101900007047491EF4D5186810BC7047E4F1FF1FFA
:1019100030B5154D83B00120AC6900F0B7F8002850
:1019200018D0E26A216BA06AFFF7D6FE002814D017
:1019300000200090019003462046AA6818302168D4
:10194000FFF7A4FA00280BD00849012008700020F6
:1019500003B030BD072003B030BD082003B030BD58
:101960000A2003B030BD0000E4F1FF1F78F0FF1F34
:10197000F7B5354886B08769164607990698FEF789
:101980001EFF012838D0002E33D03846183004907E
:101990007C6BB44200D934462246786A0799FFF737
:1019A0009BFE002843D0786A0025019500902346CD
:1019B0003969069A0498FFF769FA002834D0FBF7D2
:1019C0009FFE00280CD07969002918D0786A01950B
:1019D00000902346069A0498FFF758FA002823D06F
:1019E00006980019069007980019361B0790002EDC
:1019F000CED1002009B0F0BD0B2009B0F0BD002C05
:101A0000F5D0102C01D2254600E010252A46694663
:101A10000698FFF7F7FB002809D02A466946079881
:101A2000F6F79CFC002805D00F2009B0F0BD092076
:101A300009B0F0BD0698761B40190690079840192A
:101A40000790641BDDD1D2E7E4F1FF1F70B5FF24DE
:101A500005460134FFF744FFA04203D22846FFF7B2
:101A60003FFF0446204670BD10B5FBF741FE022043
:101A700000F00CF8072000F009F803490020087076
:101A8000FFF72EFB002010BD78F0FF1F10B5FFF709
:101A90007DFC10BD012070470025114F2C4603200E
:101AA000BC4600DF0F4E104FBC4600DF0F4F022038
:101AB000BC46B16800DF6D1CEDB2032D04D10025DA
:101AC0000120BC46B16800DF641CE4B21E2CEAD1E0
:101AD000064F00240820BC46B16800DFE3E70000A1
:101AE0007D00010060F0FF1F9500010041FF000034
:101AF00070B5194C2578032D04D0184D2E68002E92
:101B000006D006E0164A17A10020FBF7EBFB70BDDC
:101B10002860A868401C00D1A960E079032800D1A2
:101B2000E371A869904204D9E869904201D9002A7A
:101B300004D1481C06D0A868884203D0032000F0D6
:101B40002BF870BDE079984201D0032001E000201D
:101B5000AA6100F021F870BD640600204406002050
:101B60004E0200002E2E5C2E2E5C2E2E5C736F75A6
:101B70007263655C6461706C696E6B5C64726167F2
:101B80002D6E2D64726F705C7666735F6D616E6131
:101B90006765722E63000000F0B583B0054610281B
:101BA00003D0112D01D0012000E000204C4A4DA1AE
:101BB000FBF798FB584C207803280FD057490A6848
:101BC000002A12D0CB69886983420ED300280CD03A
:101BD0008B684868984208D1012007E0504A41A12B
:101BE0000020FBF77FFB03B0F0BD00206071A379FC
:101BF0000193002A02D1E279032A01D0012200E0F8
:101C000000220092002804D02279002A01D0012667
:101C100000E00026E278002A03D0002801D001204D
:101C200000E00020029008690027401C12D03B48C9
:101C30004068401C00D001201922520129A1FBF765
:101C400051FB36494A6808694969801A4002814255
:101C500000D901270321002D01D021701DE001983A
:101C600000280AD0002F01D00625F6E700980028AA
:101C7000F3D0002EF1D10425EFE702980028ECD133
:101C8000002E01D0022003E00098002802D001209D
:101C9000207011E0207803280BD16078002806D04E
:101CA000FEF7C0FF00216170002D00D105461D48E0
:101CB00005700198002896D11D4F1B491B48BC4652
:101CC00000DF184948788A78904203D1022801D170
:101CD00001208870174F1548BC4600DF03B0F0BDE7
:101CE000FE0200002E2E5C2E2E5C2E2E5C736F7575
:101CF0007263655C6461706C696E6B5C6472616771
:101D00002D6E2D64726F705C7666735F6D616E61AF
:101D10006765722E63000000640600204406002000
:101D200002030000F8F0FF1FFFFF00006C06002018
:101D3000290201007D01010070B5012514486D03E1
:101D400005601448826BC1140A438263426B0A43E4
:101D50004263114CE078F3210840E070E0785F21A5
:101D60000840E070FBF782FC0D480C49C160C91EB9
:101D70000161E0780C210843E070E07820210843FD
:101D8000E0700848056008480560012070BD00004B
:101D900080E100E00080044000B006400303000042
:101DA00000B0044080E200E000E100E00A4610B527
:101DB00001460248FBF7B8FB10BD000020190020C7
:101DC00010B501240648640304600648C17849063A
:101DD000490EC170FBF74AFC03480460012010BDA6
:101DE00080E100E000B0064000E100E0F8B5054603
:101DF000002401201F494003264608601E4FF87842
:101E00005F210840F870F878F3210840F870FBF77C
:101E10002DFC69790020012902D0022903D004E0B9
:101E20000124264600E0012401200001610008434E
:101E30003043B8702868010110480068F6F747FD84
:101E40003978400849094901C204D20E114339705A
:101E500079787870F8780C210843F87001200849E7
:101E60004003086007490860F87820210843F870AB
:101E70000120F8BD80E100E000B0064050F1FF1FF6
:101E800080E200E000E100E070B50A4601460C483F
:101E9000FBF796FB0546EFF31080C407E40F72B61C
:101EA0000748FBF7B9FA002804D00648C178802219
:101EB0001143C170002C00D162B6284670BD0000ED
:101EC0001017002000B0064010B50F4C20780028F5
:101ED00007D000202070FBF7AFF9002808D01B20A6
:101EE00010BD842209A10020FBF7FCF9022010BDDF
:101EF0006078002803D1FBF7FDFD002801D0002009
:101F000010BD212010BD0000D4F0FF1F2E2E5C2E2E
:101F10002E5C2E2E5C736F757263655C6461706CF1
:101F2000696E6B5C647261672D6E2D64726F705C9C
:101F30006961705F666C6173685F696E74662E6359
:101F400000000000F8B50F460446F6F7BCFC90A16F
:101F5000204600F0D7FB054660199AA100F0D2FB9D
:101F6000451960199BA100F0CDFB451960199DA191
:101F700000F0C8FB4519FBF7BBFB002801D09DA171
:101F800000E09DA1601900F0BDFB451960199BA1FF
:101F900000F0B8FB4519601999A100F0B3FB451991
:101FA000FBF7AEFB002801D092A100E092A16019DE
:101FB00000F0A8FB4519601990A100F0A3FB45199A
:101FC000601995A100F09EFB4519FBF7A1FB0028C5
:101FD00001D088A100E088A1601900F093FB4519A9
:101FE000601986A100F08EFB4519FBF783FD0028E0
:101FF00001D08FA600E091A6601993A100F082FBAA
:1020000045196019314600F07DFB451960197BA127
:1020100000F078FB45196019314600F073FB451953
:1020200060198DA100F06EFB4519FBF763FD0028D8
:1020300015D1FCF713FE002811D060198AA100F019
:1020400061FB4519FCF71CFE01466019042200F0F3
:1020500090FB4519601969A100F054FB4519FBF785
:102060004BFD002816D1FCF735FE002812D0601970
:1020700083A100F047FB4519FCF73EFE63190146BA
:102080000422184600F075FB451960195BA100F0A9
:1020900039FB451960197FA100F034FB451960191F
:1020A0007FA100F02FFB4519601954A100F02AFB15
:1020B0004519601985A100F025FB4519601901211A
:1020C00000F02CFB451960194CA100F01BFB4519D1
:1020D000601982A100F016FB4519601984A100F077
:1020E00011FB4519601983A100F00CFB451960191B
:1020F00082A100F007FB4519601982A100F002FBE4
:10210000451960193DA100F0FDFA4519FCF7A6FD3F
:10211000002811D060197EA100F0F4FA4519FCF7EF
:10212000C5FD62190146104600F0C2FA4519601952
:1021300032A100F0E7FA451960197AA100F0E2FA3D
:102140004519FCF7B9FD62190146104600F0B0FAD6
:102150004519601929A100F0D5FA4519601976A131
:1021600000F0D0FA784945196019896800F0D6FA6C
:102170004519601921A100F0C5FA4019201873A172
:1021800000F0C0FA39462046FBF7DCFDF8BD000040
:1021900023204441504C696E6B204669726D776113
:1021A0007265202D207365652068747470733A2FF2
:1021B0002F6D6265642E636F6D2F6461706C696E44
:1021C0006B0D0A00556E697175652049443A2040CF
:1021D000550D0A004849432049443A2040440D0A1D
:1021E000000000004175746F2052657365743A20D9
:1021F0000000000031000000300000000D0A000067
:102200004175746F6D6174696F6E20616C6C6F776E
:1022100065643A20000000004F766572666C6F7747
:1022200020646574656374696F6E3A200000000075
:10223000426F6F746C6F616465720000496E746503
:1022400072666163650000004461706C696E6B20AA
:102250004D6F64653A2000002056657273696F6E99
:102260003A2040560D0A0000426F6F746C6F616433
:1022700065722056657273696F6E3A200000000027
:10228000496E746572666163652056657273696F25
:102290006E3A2000476974205348413A20000000FC
:1022A00035623064376537653661323734333036FE
:1022B0003638306566623465336566633635376156
:1022C0003331373735373165000000004C6F6361BB
:1022D0006C204D6F64733A2000000000555342207B
:1022E000496E74657266616365733A200000000090
:1022F0004D5344002C204344430000002C20484907
:10230000440000002C205765625553420000000035
:10231000426F6F746C6F61646572204352433A2060
:1023200030780000496E74657266616365204352BF
:10233000433A20307800000052656D6F756E74204E
:10234000636F756E743A200004F1FF1F55524C3ACA
:102350002040520D0A00000010B5F8F76BFB00F0AA
:1023600085F800F00FF910BD02484078002800D031
:10237000012070478CF2FF1F10B5F8F7A5FC10BDC7
:102380000020704770B51546012820D1002B01D0E0
:10239000012B1CD10F4CA168002914D0491EA1604B
:1023A00020690D498001411840222846F6F7DAF9E4
:1023B00020690521401CF6F78AFA21616068401CFB
:1023C0006060402070BD012B01D1012020700020F1
:1023D00070BD000008F0FF1F30F3FF1FF8B5054681
:1023E0001C4814460088824201DD0020F8BD1A48CE
:1023F00000780028FAD0194E0122F2607288002A73
:1024000002D104E0002814D07288002AFAD1144FB7
:1024100022463D70781CF6F7A5F930467761002614
:10242000868044800F490978012908D87F1C4761BC
:1024300008E00020F0607061B0807080F8BD4188D5
:10244000491C41800020F9F723FA0748465501202E
:10245000F8BD0000603E01008DF2FF1FB0F2FF1FCB
:10246000701B00205E3E01009EF1FF1F002104480A
:102470000122C160016102700522426081607047E3
:1024800008F0FF1F0178832902D14078002801D08D
:10249000002070470120704770470000F8B5012503
:1024A0001746022823D1002B21D0387807281BD0CB
:1024B0001D4C606800282DD0401E6060E0681B4EF7
:1024C000800180191A463946F6F74CF9E068800118
:1024D00081193846F6F790FBE06880018019FFF714
:1024E000D1FF012804D004E0114901200870F8BD93
:1024F0000025E0680521401CF6F7E9F9E160A068D5
:10250000401CA0602078002809D0FCF75FFB002069
:10251000207004E0912207A10020FAF7E3FE28468C
:10252000FCF73EFDF8BD000008F0FF1F30F3FF1F71
:1025300004F0FF1F2E2E5C2E2E5C2E2E5C736F750A
:102540007263655C6461706C696E6B5C636D73690A
:10255000732D6461705C757362645F757365725F1F
:102560006869642E6300000010B505490020C8703A
:10257000FFF7F2FEFAF71AFCF9F784FC10BD000031
:102580008CF2FF1FB0B5094FBC4600DF084C0A4F64
:1025900060600848BC4600DFFAF7C8FE00206070A3
:1025A000A0700649A0600860B0BD0000AD07010042
:1025B000F8F0FF1F6C0600206D010100D8F2FF1F2C
:1025C000F8B51C4615460E460746FFF71FF90B489F
:1025D000006800280BD00120FCF7EAFC002C07D093
:1025E000012C04D12A4631463846FBF7BFFCF8BD22
:1025F0002A463146384600F0B3FDF8BDD8F2FF1F39
:1026000070470000FFB581B01C4616460F46FFF725
:10261000FDF815480068002823D014490020144D07
:102620008860287803281CD00120FCF7C1FC002C0E
:1026300002D0012C06D00AE032463946019800F05B
:102640007DFF04E0324639460198FBF7C9FC287843
:10265000032806D0002C04D1324639460198FBF7F6
:1026600071FD05B0F0BD0000D8F2FF1FF8F0FF1FAC
:10267000640600200548074A01780548C18000210A
:1026800001704170C1608260016170474A3E010083
:102690008CF2FF1F0100010010B5EFF31080C4079A
:1026A000E40F72B6FBF7B6F8002C00D162B610BD8D
:1026B00030B40B0E1C09124A1B07145D04700C0287
:1026C000240E1B0F2509D35C4370555D24078570CC
:1026D000240F145DC4700C04240E25092407555DD5
:1026E000240FC9B205710B09145D4471D35C09074D
:1026F0008371090F515CC17130BC08207047000024
:10270000003A010002460B780020002B05D00B5C3C
:102710001354401C0B5C002BF9D17047F3B581B00A
:102720000746002402982546002807D00A21F6F71C
:10273000CEF80021641C4D410028F7D120462843E3
:1027400001D10124002500263046311BA8410DD2BD
:102750000A210298F6F7BBF8A31B30315B1EF9542F
:10276000761C02900022301BAA41F1D3204603B010
:10277000F0BDF8B514460F460646FFF7CFFF0546F5
:10278000A0420AD2302221463046F6F777F8601B85
:1027900080193946FFF7C2FF2046F8BDF0B5002288
:1027A0000378114619434378FF252D021B02A943E4
:1027B0002B40194383782D021B04A9432B40194356
:1027C000C37804241B0619432C4B16461D695B690C
:1027D000A94209D3994214D906E0DB6CA94201D37E
:1027E00099420CD9521CD2B2244BD500EB189D6CE7
:1027F000002DF2D1DF6C002FEFD1002E3CD00C2C3D
:1028000038D81E4A926894461C4AD26896460219E5
:102810001378090A090219435378FF252D021B0278
:10282000A9432B40194393782D021B04A9432B4045
:102830001943D2780902090A12061143614501D3EE
:10284000714514D90022164606E0DB6AA94201D37D
:1028500099420CD9521CD2B2084BD500EB189D6A94
:10286000002DF2D1DF6A002FEFD1002E04D0241DFD
:102870000C2CCCD90120F0BD0020F0BDE4F1FF1FED
:1028800001783A290AD1007A302809D0322807D0B5
:10289000332805D0342803D0352801D000207047D4
:1028A00001207047FFB583B01F460398FBF7E4FC97
:1028B000FF22D2324EA1FAF715FD5A480290417A12
:1028C000007A090201435848407B41437818401E72
:1028D000F5F7FDFF00250090002F2ED0534800246F
:1028E0000569009801281FD0012600987602401E35
:1028F00001904E484E4A0069411C4300581C89B261
:10290000B04206D3FF221A324AA10020FAF7EAFCAD
:1029100002E0D154090A11544448641C0169491C5D
:10292000016101988442E4D3404C4F4A40482169F8
:1029300000F010FF2069401C20613C4E7069202887
:1029400008D3FF22E7322AA10020FAF7CBFC0020AF
:1029500007B0F0BD4101454A401C8C18706120222F
:1029600043492046F5F7FEFE0B2220460399F5F772
:10297000F9FE2777390A6177390CA177380EE077AD
:10298000280C2075000A6075A576280AE076B168E3
:10299000102908D3FF22F53215A10020FAF7A2FC76
:1029A000002007B0F0BD08460C225043324B314D99
:1029B0001D500246314DC0184560049D002D00D0C9
:1029C0009D50059A002A00D04260029A491C537A11
:1029D000157A1A02144B2A435B7B5A43009B5A43D5
:1029E0008260B1603078401C3070204607B0F0BD86
:1029F0002E2E5C2E2E5C2E2E5C736F757263655CC2
:102A00006461706C696E6B5C647261672D6E2D64BD
:102A1000726F705C7669727475616C5F66732E6339
:102A200000000000BF080020BC08002010F1FF1FBC
:102A3000BC0C00202E2E5C2E2E5C2E2E5C736F752F
:102A40007263655C6461706C696E6B5C6472616713
:102A50002D6E2D64726F705C7669727475616C5F37
:102A600066732E6300000000FFFF00003C10002092
:102A70000C3E0100FDFC0000BC0E0020F1380100FE
:102A8000C07A70471C2141180A7810464A78120211
:102A900010438A78C9781204104309060843704726
:102AA0001C2142181378194653781B021943937856
:102AB000D2781B0419431206114301D1481E7047F6
:102AC00010B5C17E807E0C0204430748017BC07AAA
:102AD0000902014305488069F5F7F9FE0249A41E81
:102AE000497B6143081810BDBC08002010F1FF1F8E
:102AF000C1727047F7B5002488B0601E088014606A
:102B000016460F4625460898FBF7B6FB002812D05C
:102B100020222146684600F099FA68460B2208995F
:102B2000F5F7C4FD002809D0002520340120A4B207
:102B300000038442ECD328460BB0F0BD6846408BBE
:102B4000388001240798240301253060EDE7000058
:102B5000F0B589B00746002502A80E462C4608901D
:102B600020222946684600F071FA6846FBF784FB8C
:102B700000281FD0684617A10B22F5F797FD002803
:102B800018D06846C07A800714D4032213A008998D
:102B9000F5F78CFD00280DD1B44209D20B2060431B
:102BA000C0190B226946F5F7DDFD641CE4B201E0B3
:102BB00001252D0320350120ADB200038542CFD37E
:102BC000074B0B2221463846F5F72BFD204609B06E
:102BD000F0BD000053454C45435452204845580031
:102BE000D931010010B50D49087DCA7C0402087B6B
:102BF000C97A000214430843002C03D107490C6A28
:102C0000002C01D0444306E00024FF22C63204A178
:102C10002046FAF767FB204610BD0000BC080020E4
:102C20002E2E5C2E2E5C2E2E5C736F757263655C8F
:102C30006461706C696E6B5C647261672D6E2D648B
:102C4000726F705C7669727475616C5F66732E6307
:102C500000000000F3B501270E467F0281B039461F
:102C60005048F5F732FE39464F48F5F72EFE4F4DE6
:102C70000024C0214E482C61F5F727FE79004D480D
:102C8000F5F723FE6C612C70AC604B48AC6168605A
:102C90003A464A494348F5F71BFB4A4848490177F9
:102CA000090A404D4177287BEA7A0102FF0111436E
:102CB000F019ED1CF5F70BFEEE1E717B424A4A43FC
:102CC000824208D9FF223A3240A10020FAF70AFBDB
:102CD000707B3D490BE04A4A5143814208D2FF22B2
:102CE0003D323AA10020FAF7FDFA707B444948438F
:102CF000B84205D32C74210A69742A49086204E099
:102D00002874010A697427490C62717BF5F7DFFDAD
:102D10003C4900024018020C3B49F282E8C92448B1
:102D2000E8C0CE688D680B68C660856003608D69F9
:102D30004B69C96985614361C161510241600161AB
:102D40001A4D0421AC61A960002110380C224A43BD
:102D500012189268AB69491CD218AA610429F5D3EC
:102D60002A4A214610482C6100F0F4FC2969284ABF
:102D7000491C0D48296100F0EDFC28696C61401C7C
:102D80000C4C2861204620222249F5F7EBFC204616
:102D90000B220199F5F7E6FC01206861FBF748F882
:102DA00003B0F0BDBC080020BC0C002010F1FF1FD8
:102DB000BC0E00203C1000204DE00000803B0100D4
:102DC00055AA00009E0A00205A1000002E2E5C2EEC
:102DD0002E5C2E2E5C736F757263655C6461706C23
:102DE000696E6B5C647261672D6E2D64726F705CCE
:102DF0007669727475616C5F66732E630000000003
:102E000091FF000080FF0000803D0100F8FF0000FE
:102E1000FFFF0000EC3D010090B40D4F04460A494D
:102E20000A48BC4600DF0B49002C0AD088780028ED
:102E300001D102208870084F0448BC4600DF90BCD6
:102E400070470020F6E70000FFFF00006C0600203E
:102E500029020100F8F0FF1F7D01010090B40C4F22
:102E600009490A48BC4600DF0A4948788A789042F6
:102E700003D1022801D101208870074F0348BC46C6
:102E800000DF90BC70470000FFFF00006C060020D0
:102E900029020100F8F0FF1F7D01010010B5FEF7C7
:102EA000B5FC0148007810BDF8F0FF1FF8B50546E5
:102EB000FEF7ACFC4A4F48494848BC4600DF494F42
:102EC0007878B97888420FD00026F6430120464A28
:102ED00046A1FAF707FA7878514C022809D0002861
:102EE0001BD001281DD025E04E4F3C48BC4600DFDA
:102EF000F8BD2078FF26F53600281BD001280AD01F
:102F0000022817D0032815D08922920037A100206B
:102F1000FAF7E8F90EE0444E0CE0B878022808D041
:102F200008E0B878022802D0002802D002E03F4E24
:102F300000E00026701C05D18D2292002BA1FAF72B
:102F4000D1F90026B868B04201D9012100E0002182
:102F5000374A904201D24019B860002905D0BD78A7
:102F60007E787D70012D07D104E02E4F1B48BC46B2
:102F700000DFF8BD0220B8700020B860294F174864
:102F8000BC4600DF0127002E15D0012E13D0022EE3
:102F900011D12078032803D0A7710020FEF7FCFD93
:102FA0002078032812D00020FF2209320FA1FAF75F
:102FB00099F900F0C3F91F4C002D09D0012D07D05D
:102FC000022DD6D1FAF7B2F92760F8BD0120EBE760
:102FD00000202060F8BD0000FFFF00006C0600200C
:102FE00029020100F8F0FF1F120200002E2E5C2EB5
:102FF0002E5C2E2E5C736F757263655C6461706C01
:10300000696E6B5C647261672D6E2D64726F705CAB
:103010007666735F6D616E616765722E6300000096
:10302000640600207D010100204E0000C40900005C
:1030300060EA0000D8F2FF1F10B5F6F757FDF6F76B
:1030400037FD10BD10B5F6F771FD10BD10B5F6F7E0
:10305000D0FD10BD024B10B5C918F6F7CAFD10BD62
:1030600000C0FE00012310B51B03C918F6F7C1FD0F
:1030700010BD70B5FF26C0B0013600243146684649
:10308000F5F723FC3501324621466846F6F748FF3E
:10309000FF340134AC42F6D340B070BDF0B5FF242C
:1030A000C1B0013421466846F5F70FFCF8206946A7
:1030B0000870FF2048708870C8701B4D2246294652
:1030C0006846F6F7EBFD21466846F5F7FEFB3D2620
:1030D000274636023A4661196846F6F721FFFF3463
:1030E0000134B442F6D339466846F5F7EEFB36A80C
:1030F000FF2226210230F5F7C1FB3A460B4968460C
:10310000F6F7CCFDFF2239466846F5F7B7FB3A469D
:1031100007496846F6F7C2FD3A4606496846F6F79B
:10312000BDFD41B0F0BD000000C0FE0000DFFE00AC
:1031300000E0FE0000E1FE0010B5F6F7AFFD10BDA7
:10314000024B10B5C918F6F7A9FD10BD00C0FE006E
:10315000012310B51B03C918F6F7E2FE10BD0000ED
:10316000F7B582B004461546002651020398F5F7DC
:10317000AAFB144900208A68002A20D931460C2273
:103180005143114A8B189B685B0AC3180093844211
:103190000CD39C420AD21F1BAF4200D32F46535878
:1031A000201A3A4603999847E419ED1B002D06D0E2
:1031B0000449761C8968F6B200988E42DED305B0C9
:1031C000F0BD000010F1FF1FBC0E00200149486057
:1031D0007047000010F1FF1F10B50B22F5F766FADB
:1031E00010BD000000B5384883B041683748FFF78C
:1031F00031FD012236490020FCF700FD0346002284
:1032000034493548FFF74EFB012231490020FCF7D5
:1032100083FC03460022314931A0FFF743FBFFF74F
:1032200011FF00280DD001231B0300222F4930A0DD
:10323000FFF738FB01239B030022304930A0FFF742
:1032400031FBFFF72BFE00280AD001222049002085
:10325000FCF76EFC034600222C492DA0FFF722FB51
:10326000194B2E4A41212E48FAF7E4FA00280DD0D6
:10327000012217490020FCF7B3FB0346002229492D
:103280002948FFF70FFB0021FFF732FC00200190D7
:103290000120C0030090FAF72FFC002811D0FF2274
:1032A000013200990198F5F759F8002809D1012257
:1032B0000749FCF7BFFC034600221C491CA0FFF78E
:1032C000F1FA03B000BD000004F1FF1F0039010056
:1032D00078060020FDFB0000F438010019FB000017
:1032E00044455441494C532054585400D5FB0000E8
:1032F000464C44495252454754585400E9FB00009B
:10330000464C4641545245475458540031FB000046
:103310004641494C202020205458540006F1FF1FFC
:1033200078080020E1F900005E3B010035FC000058
:103330004E4545445F424C205458540010B5FAF7AE
:10334000D9FB002805D0FFF7A9FD002801D1F7F728
:1033500051F9FAF7D1FB002805D0FAF7B7FA00289F
:1033600001D0F7F747F902488168491C816010BD18
:1033700004F1FF1F70B50C460546FBF7C9FB00289A
:1033800003D1FBF7BDFB002801D0012200E00022A1
:10339000002A03D1FAF7B4F9002867D0002C0BD02B
:1033A000012C63D10B223B492846F4F7D7FF0028B4
:1033B0005CD1FFF771F95DE00B2237492846F4F73D
:1033C000CDFF002841D00B2234A12846F4F7C6FFD8
:1033D000002842D00B2234A12846F4F7BFFF002872
:1033E0003CD00B2233A12846F4F7B8FF002838D090
:1033F0000B2233A12846F4F7B1FF00283AD00B2264
:1034000032A12846F4F7AAFF002830D00B2232A1BF
:103410002846F4F7A3FF00282AD00B2231A1284622
:10342000F4F79CFF002828D00B2231A12846F4F79E
:1034300095FF00282CD00B2230A12846F4F78EFFF0
:10344000002813D1FAF7E4FA14E0FAF755FB002844
:1034500010D00120FAF774FA0CE00120FAF7C4FA50
:1034600008E0B42228A10020F9F73CFF70BD01203C
:10347000FAF7C4FAFFF7F2FC70BD2F4C2068006821
:103480008047206800698047206840688047F1E7EE
:103490000120D7E75E3B01001D3901004155544F23
:1034A0005F52535443464700484152445F5253547D
:1034B0004346470041535345525420204143540052
:1034C0005245465245534820414354004155544FBC
:1034D0005F4F4E20434647004155544F5F4F46468D
:1034E0004346470045524153452020204143540064
:1034F0004F56464C5F4F4E20434647004F56464C72
:103500005F4F4646434647002E2E5C2E2E5C2E2EE5
:103510005C736F757263655C6461706C696E6B5C23
:10352000647261672D6E2D64726F705C7666735F76
:10353000757365722E630000FC390100F7B51649FA
:10354000154600268A68044682B03046002A20D9F3
:103550000C2132464A43114952189168490A4118D0
:10356000009184420CD38C420AD20F1BAF4200D38D
:103570002F465368201A3A4603999847E419ED1BE1
:10358000002D06D00449761C8968F6B200988E4258
:10359000DED305B0F0BD000010F1FF1FBC0E00200F
:1035A000F7B5064604462036307C84B015463028F0
:1035B00001D3606B32E030210F1AAF4200D31746BF
:1035C00000193A460599F5F7CDF8307CC019C1B21B
:1035D0003174302902D2002007B0F0BD05980023D5
:1035E000C0190590ED1B1A462046FAF72BFF00285C
:1035F00020D002A90022009101AB1146FAF774FF16
:103600000028E9D101986063327C2146FBF72EF84F
:103610000028E1D1317C606B401860632A4605992F
:10362000FBF724F80028D7D1606B401960631120A4
:1036300007B0F0BD192007B0F0BD0000F7B5811844
:10364000012349029B0288B0994206D9314A32A12E
:103650000020F9F747FE0BB0F0BD41024B095102C3
:1036600004914909069139495A015118029103916F
:1036700009990191002829D000260698864241D256
:1036800070010199039A4418851800902022214660
:103690002846F4F763FE002830D00B222146284646
:1036A000F4F75CFE002813D00020294F0590234634
:1036B0007F682A4602211846B84701990098085C9D
:1036C000E52807D0059800280CD017E00126D4E79C
:1036D0000120EAE723461E4C2A4664680121104671
:1036E000A0470BE02046FAF7C7FD002806D0234686
:1036F000174C2A46646800211846A0470698761C95
:103700008642BDD3049A09990298F5F72BF80BB0BD
:10371000F0BD0000BF0300002E2E5C2E2E5C2E2E6E
:103720005C736F757263655C6461706C696E6B5C11
:10373000647261672D6E2D64726F705C766972744D
:1037400075616C5F66732E63000000003C10002002
:1037500010F1FF1F10B54B000124591C6402A14257
:1037600006D3FF221A3204490020F9F7BBFD10BD31
:10377000C254120A425410BD342A0100F7B5400267
:1037800092B0570200241090002F1ED910982022CA
:103790000619314608A8FFF759FC1398202205198D
:1037A000294608A8F4F7DAFD00280BD00EA10B2259
:1037B0002846F4F77BFF002809D02022314628460E
:1037C000FFF7BAFC2034BC42E0D315B0F0BD202294
:1037D00029466846F4F7C6FF27206946C8722022AA
:1037E00031466846ECE7000053454C4543545220AF
:1037F000484558000B4610B5410252021846FFF7E3
:103800009FFC10BD0B4610B5410252021846FFF74F
:103810009FFC10BDF0B587B0002416460F46054644
:10382000039404940594FF2004AA03A90130029292
:10383000019100906B1C05AA31463846FBF7BAFD92
:1038400000280DD0022814D001281FD0042829D028
:10385000052801D00628E6D1052825D0012024E03E
:10386000049A002A27D0691C0398FAF7FFFE044641
:1038700021E0049A002A05D0691C0398FAF7F6FEA5
:10388000040018D10598361A3F18CCE7049A002A8C
:1038900004D0691C0398FAF7E9FE0446002C0AD10B
:1038A000102408E0122406E00020FF22633203A166
:1038B000F9F718FD1324204607B0F0BD2E2E5C2E1C
:1038C0002E5C2E2E5C736F757263655C6461706C28
:1038D000696E6B5C647261672D6E2D64726F705CD3
:1038E00066696C655F73747265616D2E63000000BC
:1038F0007047000043414C4C494F504548544D00DF
:103900004D494E49202020202020200090420100D7
:10391000A4420100AC420100312E31300053544129
:1039200052545F424C414354A84901004C490100A4
:103930002C490100E049010050460100F448010013
:103940006846010044480100E4470100A048010026
:10395000A8470100084A010064490100044701002A
:10396000D8460100B046010080480100C44901006A
:1039700020440100E0430100A4430100344701005A
:103980001C460100784501004045010068440100E3
:10399000444301007843010018430100B84201008C
:1039A000E8420100D8450100B8440100F444010098
:1039B000B4420100B4450100040000008800040185
:1039C000FF52070001000000102700000000000067
:1039D000CC00000098000000040000001119010054
:1039E000691A0100711901009D1801006118010098
:1039F0004D1A0100E118010041180100DC390100F5
:103A00003031323334353637383961626364656654
:103A10000000000085EE0000C91E0100B5F60000A0
:103A2000B5DB00001DDB000031F90000E1DC000027
:103A300051180100143A010000000000FFFFFFFFD1
:103A4000FFFFFFFFFFFFFFFFFFFFFFFF0000000082
:103A50000000000000000000000000000000000363
:103A6000747970653A20006572726F723A20003C7A
:103A700021646F63747970652068746D6C3E0D0A03
:103A80003C212D2D206D62656420506C6174666F41
:103A9000726D205765627369746520616E642041A0
:103AA000757468656E7469636174696F6E205368BC
:103AB0006F7274637574202D2D3E0D0A3C68746D11
:103AC0006C3E0D0A3C686561643E0D0A3C6D657490
:103AD0006120636861727365743D227574662D3868
:103AE000223E0D0A3C7469746C653E5765627369C9
:103AF00074652053686F72746375743C2F746974B5
:103B00006C653E0D0A3C2F686561643E0D0A3C629F
:103B10006F64793E0D0A3C7363726970743E0D0ADE
:103B200077696E646F772E6C6F636174696F6E2E48
:103B30007265706C6163652822405222293B0D0A30
:103B40003C2F7363726970743E0D0A3C2F626F6480
:103B5000793E0D0A3C2F68746D6C3E0D0A0041538E
:103B6000534552542020545854000000D44A0100B8
:103B7000F04A0100E04A0100E84A0100C84A010099
:103B8000EB3C904D53443053342E31000208010079
:103B9000022000501FF80100010001000000000099
:103BA00000000000000029741902274441504C49CC
:103BB0004E4B2D444E4446415431362020200000C7
:103BC00000000000000000000000000000000000F5
:103BD00000000000000000000000000000000000E5
:103BE00000000000000000000000000000000000D5
:103BF00000000000000000000000000000000000C5
:103C000000000000000000000000000000000000B4
:103C100000000000000000000000000000000000A4
:103C20000000000000000000000000000000000094
:103C30000000000000000000000000000000000084
:103C40000000000000000000000000000000000074
:103C50000000000000000000000000000000000064
:103C60000000000000000000000000000000000054
:103C70000000000000000000000000000000000044
:103C80000000000000000000000000000000000034
:103C90000000000000000000000000000000000024
:103CA0000000000000000000000000000000000014
:103CB0000000000000000000000000000000000004
:103CC00000000000000000000000000000000000F4
:103CD00000000000000000000000000000000000E4
:103CE00000000000000000000000000000000000D4
:103CF00000000000000000000000000000000000C4
:103D000000000000000000000000000000000000B3
:103D100000000000000000000000000000000000A3
:103D20000000000000000000000000000000000093
:103D30000000000000000000000000000000000083
:103D40000000000000000000000000000000000073
:103D50000000000000000000000000000000000063
:103D60000000000000000000000000000000000053
:103D70000000000000000000000000000000000043
:103D8000C1FC0000F138010000020000BDF9000094
:103D9000F138010000000000BDF90000F138010019
:103DA0000000000039F900003D3601000004000069
:103DB0009DFC0000F13801000002000075FC0000CD
:103DC000F53701000000000075FC0000F13801002B
:103DD0000000000061FC00007D37010000100000C1
:103DE00089FC00000538010000B0FE000000000062
:103DF000000000000000002800000000000000009B
:103E00000000418EBB3200000000000000000000F6
:103E10000000000000000000000000007648764826
:103E20000000DC837648000000000000080010005D
:103E3000180020003000400060008000C000000139
:103E400080010002000300040006000001000500DC
:103E50004003040101000100400040004000010156
:103E60004000400000020200400000024000010249
:103E700004044000400040004000212065D10000C3
:103E8000000000000000000071D1000000000000F0
:103E900085AD000065BA000045C20000FF83000048
:103EA000C9A90000000000000000000000000000A0
:103EB0000000000000000000000000000000000002
:103EC00000000000000000000000000000000000F2
:103ED000BFAC000000000000000000000600FF0969
:103EE00001A101150026FF00750895400901810216
:103EF00095400901910295010901B102C00021001C
:103F00006B0012011002EF020140280D04020010A4
:103F10000102030100000A00000000000306AA00DD
:103F2000080002000400A0001400030057494E5589
:103F30005342000000000000000000008400040064
:103F400007002A00440065007600690063006500F0
:103F500049006E0074006500720066006100630035
:103F60006500470055004900440073000000500000
:103F70007B00390032004300450036003400360033
:103F800032002D0039004300370037002D00340087
:103F90003600460045002D00390033003300420052
:103FA0002D0033003100430042003900430035004A
:103FB000410041003300420039007D000000000054
:103FC000050F3900021810050038B60834A909A0F9
:103FD000478BFDA0768815B665000121001C1005F1
:103FE00000DF60DDD88945C74C9CD2659D9E648A00
:103FF0009F00000306AA00200009028B00050100B3
:1040000080FA0904000002080650080705820240F1
:10401000000007050202400000080B010202020135
:104020000409040100010202010405240010010535
:104030002401030204240206052406010207058365
:104040000310002009040200020A0000050705040D
:10405000024000000705840240000009040300023A
:10406000030000060921000100012221000705814B
:10407000034000010705010340000109040400009A
:10408000FF030007000000000403090408034100C7
:1040900052004D00300342004200430020006D00FA
:1040A0006900630072006F003A00620069007400EA
:1040B000200043004D005300490053002D004400F0
:1040C000410050001A033000300030003100410040
:1040D000300030003000300030003000300022036B
:1040E0006D006200650064002000530065007200EE
:1040F000690061006C00200050006F0072007400C5
:1041000022036D006200650064002000530065001A
:104110007200690061006C00200050006F007200A6
:104120007400140343004D005300490053002D0058
:104130004400410050002403570065006200550010
:10414000530042003A00200043004D005300490054
:1041500053002D004400410050001003550053004F
:1041600042005F004D0053004300000000000000CB
:104170000001010000BE0AE00D782D066840082409
:10418000400000D35840641EFAD1491C521E002A38
:10419000F2D17047002070470020704770B5264C60
:1041A000022060600120E060244D2868C00702D032
:1041B0000020606070BD00F02CF8F6E770B51E4C72
:1041C000022161601E49884202D30120606100E043
:1041D000A0601A4D00F01DF82868C007FAD0002032
:1041E000606070BDF8B505468E081348012114467D
:1041F0004160124F01CC01C53868C00706D0761E59
:10420000F8D10D48002141600846F8BD00F001F8E2
:10421000F2E70C4840680006000E0BD00A494968D6
:10422000002907D009490A4AC30700D00A60091DBE
:104230004008F9D17047000000E5014000E401406A
:10424000001000100004014000050140000601407C
:104250003546526E0000000021000020250000209D
:10426000290000204900002071000020000000000B
:10427000010000207001002000100020000200203A
:104280000000002050010000744101000002000005
:1042900068747470733A2F2F63616C6C696F70650A
:1042A0002E63630039393030000000003939303175
:1042B0000000000000000000496E206170706C6911
:1042C000636174696F6E2070726F6772616D6D6982
:1042D0006E6720736563746F722065726173652009
:1042E0006661696C65642E00496E206170706C694E
:1042F000636174696F6E2070726F6772616D6D6952
:104300006E67206D617373206572617365206661ED
:10431000696C65642E000000496E206170706C69E4
:10432000636174696F6E2070726F6772616D6D6921
:104330006E67207772697465206661696C65642EAA
:1043400000000000496E206170706C6963617469DF
:104350006F6E2070726F6772616D6D696E67206934
:104360006E697469616C697A6174696F6E206661E7
:10437000696C65642E000000496E206170706C6984
:10438000636174696F6E2070726F6772616D6D69C1
:104390006E6720756E696E6974206661696C65640C
:1043A0002E000000546865206865782066696C6599
:1043B0002063616E6E6F742062652070726F677229
:1043C000616D6D65642E204C6F676963206661695D
:1043D0006C757265206F636375727265642E000080
:1043E000546865206865782066696C652063616E35
:1043F0006E6F74206265206465636F6465642E204F
:10440000506172736572206C6F67696320666169C1
:104410006C757265206F636375727265642E00003F
:10442000546865206865782066696C652063616EF4
:104430006E6F74206265206465636F6465642E200E
:10444000436865636B73756D2063616C63756C6144
:1044500074696F6E206661696C757265206F636345
:1044600075727265642E0000546865206170706C0E
:1044700069636174696F6E2066696C6520666F722E
:104480006D617420697320756E6B6E6F776E20613D
:104490006E642063616E6E6F74206265207061725D
:1044A00073656420616E642F6F722070726F636534
:1044B000737365642E000000496E206170706C6932
:1044C000636174696F6E2070726F6772616D6D6980
:1044D0006E67206E6F7420737570706F7274656490
:1044E000206F6E2074686973206465766963652E39
:1044F00000000000496E206170706C69636174692E
:104500006F6E2070726F6772616D6D696E67206685
:1045100061696C65642062656361757365207468A8
:1045200065207570646174652073656E74207761B1
:104530007320696E636F6D706C6574652E0000008A
:10454000546865207374617274696E672061646475
:104550007265737320666F722074686520696E746B
:104560006572666163652075706461746520697346
:104570002077726F6E672E005468652073746172C5
:1045800074696E67206164647265737320666F720C
:104590002074686520626F6F746C6F61646572204F
:1045A0007570646174652069732077726F6E672E11
:1045B0000000000054686520626F6F746C6F616466
:1045C00065722043524320646964206E6F742070CA
:1045D0006173732E00000000496E206170706C6979
:1045E000636174696F6E2070726F6772616D6D695F
:1045F0006E672061626F72746564206475652074F3
:104600006F20616E206F7574206F6620626F756E0B
:10461000647320616464726573732E00546865204E
:104620006865782066696C65206F666673657420BE
:104630006C6F6164206164647265737320697320B8
:104640006E6F7420636F72726563742E00000000D9
:10465000546865207472616E736665722074696D4A
:104660006564206F75742E0046696C652073656EF5
:1046700074206F7574206F66206F7264657220629B
:10468000792050432E20546172676574206D6967EC
:104690006874206E6F742062652070726F6772613B
:1046A0006D6D656420636F72726563746C792E0042
:1046B000466C61736820616C676F726974686D2005
:1046C000777269746520636F6D6D616E6420464119
:1046D000494C555245000000466C61736820616C7E
:1046E000676F726974686D20657261736520616CB3
:1046F0006C20636F6D6D616E64204641494C55526C
:1047000045000000466C61736820616C676F7269D8
:1047100074686D20657261736520736563746F7270
:1047200020636F6D6D616E64204641494C55524562
:1047300000000000546865206865782066696C6533
:1047400020796F752064726F707065642069736E74
:10475000277420636F6D70617469626C652077697E
:1047600074682074686973206D6F6465206F7220AF
:104770006465766963652E2041726520796F7520C6
:10478000696E204D41494E54454E414E4345206D82
:104790006F64653F205365652048454C5020464175
:1047A000512E48544D00000054686520696E7465B0
:1047B0007266616365206669726D77617265204615
:1047C00041494C454420746F20696E697469616C7D
:1047D000697A652074686520746172676574204D1C
:1047E0004355000054686520696E746572666163A4
:1047F00065206669726D77617265204641494C4556
:104800004420746F20646F776E6C6F6164207468ED
:104810006520666C6173682070726F6772616D6D80
:10482000696E6720616C676F726974686D7320745C
:104830006F2074686520746172676574204D4355FC
:104840000000000054686520696E746572666163DB
:1048500065206669726D77617265204641494C45F5
:104860004420746F2072657365742F68616C7420C6
:1048700074686520746172676574204D435500004B
:10488000456E64206F662073747265616D20686187
:1048900073206265656E20726561636865640000FF
:1048A00054686520696E7465726661636520666927
:1048B000726D77617265204641494C454420746FA2
:1048C00020646F776E6C6F61642074686520666C1D
:1048D000617368206461746120636F6E74656E74C7
:1048E0007320746F2062652070726F6772616D6DE6
:1048F00065640000506F737369626C65206D697345
:104900006D61746368206265747765656E206669A1
:104910006C652073697A6520616E642073697A65BD
:104920002070726F6772616D6D656400416E206901
:104930006E7465726E616C206572726F7220686150
:1049400073206F636375727265640000416E206549
:1049500072726F7220686173206F63637572726523
:104960006400000054686520696E74657266616356
:1049700065206669726D77617265204641494C45D4
:104980004420746F20756E6C6F636B2074686520B3
:1049900074617267657420666F722070726F6772DF
:1049A000616D6D696E6700004F7065726174696F4B
:1049B0006E20776173207375636365737366756CBE
:1049C00000000000456E64206F662073747265619C
:1049D0006D20697320756E6B6E6F776E000000003E
:1049E000416E206572726F72206F636375727265BB
:1049F0006420647572696E672074686520747261E2
:104A00006E7366657200000054686520696E746597
:104A10007266616365206669726D776172652041B7
:104A2000424F525445442070726F6772616D6D69D8
:104A30006E672E20496D61676520697320747279F5
:104A4000696E6720746F2073657420736563757277
:104A50006974792062697473000000004120626FFC
:104A60006F746C6F61646572207570646174652029
:104A70007761732073746172746564206275742049
:104A8000756E61626C6520746F20636F6D706C650C
:104A900074652E0D0A52656C6F6164207468652020
:104AA000626F6F746C6F6164657220746F206669E9
:104AB000782074686973206572726F72206D6573F7
:104AC000736167652E0D0A00696E746572666163B5
:104AD00065000000696E7465726E616C0000000014
:104AE0007573657200000000746172676574000080
:104AF0007472616E7369656E740000004D424544C6
:104B00002020202056465320202020202020202016
:104B100020202020302E3100384B010000F0FF1FF4
:104B2000180300009E8B0000D04B010018F3FF1FFC
:104B30003835000004810000041AB442011808014D
:104B4000010206020208012A04052F0101060606D9
:104B500004017A1001051F019996970B1901016351
:104B60008123FDDA23F5F214A1350123E1D61B0FD1
:104B7000DB141910141538011AE9100163024504F9
:104B8000176CDC02FC4A0140292C03016F732E6D67
:104B90006265642E636F6D2F7765627573622F6C2B
:104BA000616E64696E672D706167652F3F6269642D
:104BB0003DCA132C01211A5501E10A20FFDABA017E
:104BC000E7122012408D205842011701FF0110000A
:104BD000FFFFFFFFFFFFFFFFFFFFFFFFFFFFFFFFE5
:104BE000FFFFFFFFFFFFFFFFFFFFFFFFFFFFFFFFD5
:104BF000FFFFFFFFFFFFFFFFFFFFFFFFFFFFFFFFC5
:104C0000FFFFFFFFFFFFFFFFFFFFFFFFFFFFFFFFB4
:10FBF000FFFFFFFFFFFFFFFFFFFFFFFF0FD121B759
:00000001FF
